
lab_00.elf:     file format elf32-littlearm

Sections:
Idx Name          Size      VMA       LMA       File off  Algn
  0 .isr_vector   00000198  08000000  08000000  00010000  2**0
                  CONTENTS, ALLOC, LOAD, READONLY, DATA
  1 .text         00001144  08000198  08000198  00010198  2**2
                  CONTENTS, ALLOC, LOAD, READONLY, CODE
  2 .rodata       00000018  080012dc  080012dc  000112dc  2**0
                  CONTENTS, ALLOC, LOAD, READONLY, DATA
  3 .ARM          00000008  080012f4  080012f4  000112f4  2**2
                  CONTENTS, ALLOC, LOAD, READONLY, DATA
  4 .init_array   00000004  080012fc  080012fc  000112fc  2**2
                  CONTENTS, ALLOC, LOAD, DATA
  5 .fini_array   00000004  08001300  08001300  00011300  2**2
                  CONTENTS, ALLOC, LOAD, DATA
  6 .data         0000000c  20000000  08001304  00020000  2**2
                  CONTENTS, ALLOC, LOAD, DATA
  7 .bss          00000060  2000000c  08001310  0002000c  2**2
                  ALLOC
  8 ._user_heap_stack 00000600  2000006c  08001310  0002006c  2**0
                  ALLOC
  9 .ARM.attributes 00000030  00000000  00000000  0002000c  2**0
                  CONTENTS, READONLY
 10 .debug_info   00005ed6  00000000  00000000  0002003c  2**0
                  CONTENTS, READONLY, DEBUGGING
 11 .debug_abbrev 00001392  00000000  00000000  00025f12  2**0
                  CONTENTS, READONLY, DEBUGGING
 12 .debug_loc    00002116  00000000  00000000  000272a4  2**0
                  CONTENTS, READONLY, DEBUGGING
 13 .debug_aranges 000004d8  00000000  00000000  000293c0  2**3
                  CONTENTS, READONLY, DEBUGGING
 14 .debug_ranges 000005c0  00000000  00000000  00029898  2**3
                  CONTENTS, READONLY, DEBUGGING
 15 .debug_line   0000268a  00000000  00000000  00029e58  2**0
                  CONTENTS, READONLY, DEBUGGING
 16 .debug_str    00001e0e  00000000  00000000  0002c4e2  2**0
                  CONTENTS, READONLY, DEBUGGING
 17 .comment      0000007c  00000000  00000000  0002e2f0  2**0
                  CONTENTS, READONLY
 18 .debug_frame  00000c30  00000000  00000000  0002e36c  2**2
                  CONTENTS, READONLY, DEBUGGING

Disassembly of section .text:

08000198 <__do_global_dtors_aux>:
 8000198:	b510      	push	{r4, lr}
 800019a:	4c05      	ldr	r4, [pc, #20]	; (80001b0 <__do_global_dtors_aux+0x18>)
 800019c:	7823      	ldrb	r3, [r4, #0]
 800019e:	b933      	cbnz	r3, 80001ae <__do_global_dtors_aux+0x16>
 80001a0:	4b04      	ldr	r3, [pc, #16]	; (80001b4 <__do_global_dtors_aux+0x1c>)
 80001a2:	b113      	cbz	r3, 80001aa <__do_global_dtors_aux+0x12>
 80001a4:	4804      	ldr	r0, [pc, #16]	; (80001b8 <__do_global_dtors_aux+0x20>)
 80001a6:	f3af 8000 	nop.w
 80001aa:	2301      	movs	r3, #1
 80001ac:	7023      	strb	r3, [r4, #0]
 80001ae:	bd10      	pop	{r4, pc}
 80001b0:	2000000c 	.word	0x2000000c
 80001b4:	00000000 	.word	0x00000000
 80001b8:	080012c4 	.word	0x080012c4

080001bc <frame_dummy>:
 80001bc:	b508      	push	{r3, lr}
 80001be:	4b03      	ldr	r3, [pc, #12]	; (80001cc <frame_dummy+0x10>)
 80001c0:	b11b      	cbz	r3, 80001ca <frame_dummy+0xe>
 80001c2:	4903      	ldr	r1, [pc, #12]	; (80001d0 <frame_dummy+0x14>)
 80001c4:	4803      	ldr	r0, [pc, #12]	; (80001d4 <frame_dummy+0x18>)
 80001c6:	f3af 8000 	nop.w
 80001ca:	bd08      	pop	{r3, pc}
 80001cc:	00000000 	.word	0x00000000
 80001d0:	20000010 	.word	0x20000010
 80001d4:	080012c4 	.word	0x080012c4

080001d8 <__aeabi_uldivmod>:
 80001d8:	b953      	cbnz	r3, 80001f0 <__aeabi_uldivmod+0x18>
 80001da:	b94a      	cbnz	r2, 80001f0 <__aeabi_uldivmod+0x18>
 80001dc:	2900      	cmp	r1, #0
 80001de:	bf08      	it	eq
 80001e0:	2800      	cmpeq	r0, #0
 80001e2:	bf1c      	itt	ne
 80001e4:	f04f 31ff 	movne.w	r1, #4294967295
 80001e8:	f04f 30ff 	movne.w	r0, #4294967295
 80001ec:	f000 b97a 	b.w	80004e4 <__aeabi_idiv0>
 80001f0:	f1ad 0c08 	sub.w	ip, sp, #8
 80001f4:	e96d ce04 	strd	ip, lr, [sp, #-16]!
 80001f8:	f000 f806 	bl	8000208 <__udivmoddi4>
 80001fc:	f8dd e004 	ldr.w	lr, [sp, #4]
 8000200:	e9dd 2302 	ldrd	r2, r3, [sp, #8]
 8000204:	b004      	add	sp, #16
 8000206:	4770      	bx	lr

08000208 <__udivmoddi4>:
 8000208:	e92d 47f0 	stmdb	sp!, {r4, r5, r6, r7, r8, r9, sl, lr}
 800020c:	468c      	mov	ip, r1
 800020e:	460d      	mov	r5, r1
 8000210:	4604      	mov	r4, r0
 8000212:	9e08      	ldr	r6, [sp, #32]
 8000214:	2b00      	cmp	r3, #0
 8000216:	d151      	bne.n	80002bc <__udivmoddi4+0xb4>
 8000218:	428a      	cmp	r2, r1
 800021a:	4617      	mov	r7, r2
 800021c:	d96d      	bls.n	80002fa <__udivmoddi4+0xf2>
 800021e:	fab2 fe82 	clz	lr, r2
 8000222:	f1be 0f00 	cmp.w	lr, #0
 8000226:	d00b      	beq.n	8000240 <__udivmoddi4+0x38>
 8000228:	f1ce 0c20 	rsb	ip, lr, #32
 800022c:	fa01 f50e 	lsl.w	r5, r1, lr
 8000230:	fa20 fc0c 	lsr.w	ip, r0, ip
 8000234:	fa02 f70e 	lsl.w	r7, r2, lr
 8000238:	ea4c 0c05 	orr.w	ip, ip, r5
 800023c:	fa00 f40e 	lsl.w	r4, r0, lr
 8000240:	ea4f 4a17 	mov.w	sl, r7, lsr #16
 8000244:	0c25      	lsrs	r5, r4, #16
 8000246:	fbbc f8fa 	udiv	r8, ip, sl
 800024a:	fa1f f987 	uxth.w	r9, r7
 800024e:	fb0a cc18 	mls	ip, sl, r8, ip
 8000252:	ea45 450c 	orr.w	r5, r5, ip, lsl #16
 8000256:	fb08 f309 	mul.w	r3, r8, r9
 800025a:	42ab      	cmp	r3, r5
 800025c:	d90a      	bls.n	8000274 <__udivmoddi4+0x6c>
 800025e:	19ed      	adds	r5, r5, r7
 8000260:	f108 32ff 	add.w	r2, r8, #4294967295
 8000264:	f080 8123 	bcs.w	80004ae <__udivmoddi4+0x2a6>
 8000268:	42ab      	cmp	r3, r5
 800026a:	f240 8120 	bls.w	80004ae <__udivmoddi4+0x2a6>
 800026e:	f1a8 0802 	sub.w	r8, r8, #2
 8000272:	443d      	add	r5, r7
 8000274:	1aed      	subs	r5, r5, r3
 8000276:	b2a4      	uxth	r4, r4
 8000278:	fbb5 f0fa 	udiv	r0, r5, sl
 800027c:	fb0a 5510 	mls	r5, sl, r0, r5
 8000280:	ea44 4405 	orr.w	r4, r4, r5, lsl #16
 8000284:	fb00 f909 	mul.w	r9, r0, r9
 8000288:	45a1      	cmp	r9, r4
 800028a:	d909      	bls.n	80002a0 <__udivmoddi4+0x98>
 800028c:	19e4      	adds	r4, r4, r7
 800028e:	f100 33ff 	add.w	r3, r0, #4294967295
 8000292:	f080 810a 	bcs.w	80004aa <__udivmoddi4+0x2a2>
 8000296:	45a1      	cmp	r9, r4
 8000298:	f240 8107 	bls.w	80004aa <__udivmoddi4+0x2a2>
 800029c:	3802      	subs	r0, #2
 800029e:	443c      	add	r4, r7
 80002a0:	eba4 0409 	sub.w	r4, r4, r9
 80002a4:	ea40 4008 	orr.w	r0, r0, r8, lsl #16
 80002a8:	2100      	movs	r1, #0
 80002aa:	2e00      	cmp	r6, #0
 80002ac:	d061      	beq.n	8000372 <__udivmoddi4+0x16a>
 80002ae:	fa24 f40e 	lsr.w	r4, r4, lr
 80002b2:	2300      	movs	r3, #0
 80002b4:	6034      	str	r4, [r6, #0]
 80002b6:	6073      	str	r3, [r6, #4]
 80002b8:	e8bd 87f0 	ldmia.w	sp!, {r4, r5, r6, r7, r8, r9, sl, pc}
 80002bc:	428b      	cmp	r3, r1
 80002be:	d907      	bls.n	80002d0 <__udivmoddi4+0xc8>
 80002c0:	2e00      	cmp	r6, #0
 80002c2:	d054      	beq.n	800036e <__udivmoddi4+0x166>
 80002c4:	2100      	movs	r1, #0
 80002c6:	e886 0021 	stmia.w	r6, {r0, r5}
 80002ca:	4608      	mov	r0, r1
 80002cc:	e8bd 87f0 	ldmia.w	sp!, {r4, r5, r6, r7, r8, r9, sl, pc}
 80002d0:	fab3 f183 	clz	r1, r3
 80002d4:	2900      	cmp	r1, #0
 80002d6:	f040 808e 	bne.w	80003f6 <__udivmoddi4+0x1ee>
 80002da:	42ab      	cmp	r3, r5
 80002dc:	d302      	bcc.n	80002e4 <__udivmoddi4+0xdc>
 80002de:	4282      	cmp	r2, r0
 80002e0:	f200 80fa 	bhi.w	80004d8 <__udivmoddi4+0x2d0>
 80002e4:	1a84      	subs	r4, r0, r2
 80002e6:	eb65 0503 	sbc.w	r5, r5, r3
 80002ea:	2001      	movs	r0, #1
 80002ec:	46ac      	mov	ip, r5
 80002ee:	2e00      	cmp	r6, #0
 80002f0:	d03f      	beq.n	8000372 <__udivmoddi4+0x16a>
 80002f2:	e886 1010 	stmia.w	r6, {r4, ip}
 80002f6:	e8bd 87f0 	ldmia.w	sp!, {r4, r5, r6, r7, r8, r9, sl, pc}
 80002fa:	b912      	cbnz	r2, 8000302 <__udivmoddi4+0xfa>
 80002fc:	2701      	movs	r7, #1
 80002fe:	fbb7 f7f2 	udiv	r7, r7, r2
 8000302:	fab7 fe87 	clz	lr, r7
 8000306:	f1be 0f00 	cmp.w	lr, #0
 800030a:	d134      	bne.n	8000376 <__udivmoddi4+0x16e>
 800030c:	1beb      	subs	r3, r5, r7
 800030e:	0c3a      	lsrs	r2, r7, #16
 8000310:	fa1f fc87 	uxth.w	ip, r7
 8000314:	2101      	movs	r1, #1
 8000316:	fbb3 f8f2 	udiv	r8, r3, r2
 800031a:	0c25      	lsrs	r5, r4, #16
 800031c:	fb02 3318 	mls	r3, r2, r8, r3
 8000320:	ea45 4503 	orr.w	r5, r5, r3, lsl #16
 8000324:	fb0c f308 	mul.w	r3, ip, r8
 8000328:	42ab      	cmp	r3, r5
 800032a:	d907      	bls.n	800033c <__udivmoddi4+0x134>
 800032c:	19ed      	adds	r5, r5, r7
 800032e:	f108 30ff 	add.w	r0, r8, #4294967295
 8000332:	d202      	bcs.n	800033a <__udivmoddi4+0x132>
 8000334:	42ab      	cmp	r3, r5
 8000336:	f200 80d1 	bhi.w	80004dc <__udivmoddi4+0x2d4>
 800033a:	4680      	mov	r8, r0
 800033c:	1aed      	subs	r5, r5, r3
 800033e:	b2a3      	uxth	r3, r4
 8000340:	fbb5 f0f2 	udiv	r0, r5, r2
 8000344:	fb02 5510 	mls	r5, r2, r0, r5
 8000348:	ea43 4405 	orr.w	r4, r3, r5, lsl #16
 800034c:	fb0c fc00 	mul.w	ip, ip, r0
 8000350:	45a4      	cmp	ip, r4
 8000352:	d907      	bls.n	8000364 <__udivmoddi4+0x15c>
 8000354:	19e4      	adds	r4, r4, r7
 8000356:	f100 33ff 	add.w	r3, r0, #4294967295
 800035a:	d202      	bcs.n	8000362 <__udivmoddi4+0x15a>
 800035c:	45a4      	cmp	ip, r4
 800035e:	f200 80b8 	bhi.w	80004d2 <__udivmoddi4+0x2ca>
 8000362:	4618      	mov	r0, r3
 8000364:	eba4 040c 	sub.w	r4, r4, ip
 8000368:	ea40 4008 	orr.w	r0, r0, r8, lsl #16
 800036c:	e79d      	b.n	80002aa <__udivmoddi4+0xa2>
 800036e:	4631      	mov	r1, r6
 8000370:	4630      	mov	r0, r6
 8000372:	e8bd 87f0 	ldmia.w	sp!, {r4, r5, r6, r7, r8, r9, sl, pc}
 8000376:	f1ce 0420 	rsb	r4, lr, #32
 800037a:	fa05 f30e 	lsl.w	r3, r5, lr
 800037e:	fa07 f70e 	lsl.w	r7, r7, lr
 8000382:	fa20 f804 	lsr.w	r8, r0, r4
 8000386:	0c3a      	lsrs	r2, r7, #16
 8000388:	fa25 f404 	lsr.w	r4, r5, r4
 800038c:	ea48 0803 	orr.w	r8, r8, r3
 8000390:	fbb4 f1f2 	udiv	r1, r4, r2
 8000394:	ea4f 4518 	mov.w	r5, r8, lsr #16
 8000398:	fb02 4411 	mls	r4, r2, r1, r4
 800039c:	fa1f fc87 	uxth.w	ip, r7
 80003a0:	ea45 4504 	orr.w	r5, r5, r4, lsl #16
 80003a4:	fb01 f30c 	mul.w	r3, r1, ip
 80003a8:	42ab      	cmp	r3, r5
 80003aa:	fa00 f40e 	lsl.w	r4, r0, lr
 80003ae:	d909      	bls.n	80003c4 <__udivmoddi4+0x1bc>
 80003b0:	19ed      	adds	r5, r5, r7
 80003b2:	f101 30ff 	add.w	r0, r1, #4294967295
 80003b6:	f080 808a 	bcs.w	80004ce <__udivmoddi4+0x2c6>
 80003ba:	42ab      	cmp	r3, r5
 80003bc:	f240 8087 	bls.w	80004ce <__udivmoddi4+0x2c6>
 80003c0:	3902      	subs	r1, #2
 80003c2:	443d      	add	r5, r7
 80003c4:	1aeb      	subs	r3, r5, r3
 80003c6:	fa1f f588 	uxth.w	r5, r8
 80003ca:	fbb3 f0f2 	udiv	r0, r3, r2
 80003ce:	fb02 3310 	mls	r3, r2, r0, r3
 80003d2:	ea45 4503 	orr.w	r5, r5, r3, lsl #16
 80003d6:	fb00 f30c 	mul.w	r3, r0, ip
 80003da:	42ab      	cmp	r3, r5
 80003dc:	d907      	bls.n	80003ee <__udivmoddi4+0x1e6>
 80003de:	19ed      	adds	r5, r5, r7
 80003e0:	f100 38ff 	add.w	r8, r0, #4294967295
 80003e4:	d26f      	bcs.n	80004c6 <__udivmoddi4+0x2be>
 80003e6:	42ab      	cmp	r3, r5
 80003e8:	d96d      	bls.n	80004c6 <__udivmoddi4+0x2be>
 80003ea:	3802      	subs	r0, #2
 80003ec:	443d      	add	r5, r7
 80003ee:	1aeb      	subs	r3, r5, r3
 80003f0:	ea40 4101 	orr.w	r1, r0, r1, lsl #16
 80003f4:	e78f      	b.n	8000316 <__udivmoddi4+0x10e>
 80003f6:	f1c1 0720 	rsb	r7, r1, #32
 80003fa:	fa22 f807 	lsr.w	r8, r2, r7
 80003fe:	408b      	lsls	r3, r1
 8000400:	fa05 f401 	lsl.w	r4, r5, r1
 8000404:	ea48 0303 	orr.w	r3, r8, r3
 8000408:	fa20 fe07 	lsr.w	lr, r0, r7
 800040c:	ea4f 4c13 	mov.w	ip, r3, lsr #16
 8000410:	40fd      	lsrs	r5, r7
 8000412:	ea4e 0e04 	orr.w	lr, lr, r4
 8000416:	fbb5 f9fc 	udiv	r9, r5, ip
 800041a:	ea4f 441e 	mov.w	r4, lr, lsr #16
 800041e:	fb0c 5519 	mls	r5, ip, r9, r5
 8000422:	fa1f f883 	uxth.w	r8, r3
 8000426:	ea44 4505 	orr.w	r5, r4, r5, lsl #16
 800042a:	fb09 f408 	mul.w	r4, r9, r8
 800042e:	42ac      	cmp	r4, r5
 8000430:	fa02 f201 	lsl.w	r2, r2, r1
 8000434:	fa00 fa01 	lsl.w	sl, r0, r1
 8000438:	d908      	bls.n	800044c <__udivmoddi4+0x244>
 800043a:	18ed      	adds	r5, r5, r3
 800043c:	f109 30ff 	add.w	r0, r9, #4294967295
 8000440:	d243      	bcs.n	80004ca <__udivmoddi4+0x2c2>
 8000442:	42ac      	cmp	r4, r5
 8000444:	d941      	bls.n	80004ca <__udivmoddi4+0x2c2>
 8000446:	f1a9 0902 	sub.w	r9, r9, #2
 800044a:	441d      	add	r5, r3
 800044c:	1b2d      	subs	r5, r5, r4
 800044e:	fa1f fe8e 	uxth.w	lr, lr
 8000452:	fbb5 f0fc 	udiv	r0, r5, ip
 8000456:	fb0c 5510 	mls	r5, ip, r0, r5
 800045a:	ea4e 4405 	orr.w	r4, lr, r5, lsl #16
 800045e:	fb00 f808 	mul.w	r8, r0, r8
 8000462:	45a0      	cmp	r8, r4
 8000464:	d907      	bls.n	8000476 <__udivmoddi4+0x26e>
 8000466:	18e4      	adds	r4, r4, r3
 8000468:	f100 35ff 	add.w	r5, r0, #4294967295
 800046c:	d229      	bcs.n	80004c2 <__udivmoddi4+0x2ba>
 800046e:	45a0      	cmp	r8, r4
 8000470:	d927      	bls.n	80004c2 <__udivmoddi4+0x2ba>
 8000472:	3802      	subs	r0, #2
 8000474:	441c      	add	r4, r3
 8000476:	ea40 4009 	orr.w	r0, r0, r9, lsl #16
 800047a:	eba4 0408 	sub.w	r4, r4, r8
 800047e:	fba0 8902 	umull	r8, r9, r0, r2
 8000482:	454c      	cmp	r4, r9
 8000484:	46c6      	mov	lr, r8
 8000486:	464d      	mov	r5, r9
 8000488:	d315      	bcc.n	80004b6 <__udivmoddi4+0x2ae>
 800048a:	d012      	beq.n	80004b2 <__udivmoddi4+0x2aa>
 800048c:	b156      	cbz	r6, 80004a4 <__udivmoddi4+0x29c>
 800048e:	ebba 030e 	subs.w	r3, sl, lr
 8000492:	eb64 0405 	sbc.w	r4, r4, r5
 8000496:	fa04 f707 	lsl.w	r7, r4, r7
 800049a:	40cb      	lsrs	r3, r1
 800049c:	431f      	orrs	r7, r3
 800049e:	40cc      	lsrs	r4, r1
 80004a0:	6037      	str	r7, [r6, #0]
 80004a2:	6074      	str	r4, [r6, #4]
 80004a4:	2100      	movs	r1, #0
 80004a6:	e8bd 87f0 	ldmia.w	sp!, {r4, r5, r6, r7, r8, r9, sl, pc}
 80004aa:	4618      	mov	r0, r3
 80004ac:	e6f8      	b.n	80002a0 <__udivmoddi4+0x98>
 80004ae:	4690      	mov	r8, r2
 80004b0:	e6e0      	b.n	8000274 <__udivmoddi4+0x6c>
 80004b2:	45c2      	cmp	sl, r8
 80004b4:	d2ea      	bcs.n	800048c <__udivmoddi4+0x284>
 80004b6:	ebb8 0e02 	subs.w	lr, r8, r2
 80004ba:	eb69 0503 	sbc.w	r5, r9, r3
 80004be:	3801      	subs	r0, #1
 80004c0:	e7e4      	b.n	800048c <__udivmoddi4+0x284>
 80004c2:	4628      	mov	r0, r5
 80004c4:	e7d7      	b.n	8000476 <__udivmoddi4+0x26e>
 80004c6:	4640      	mov	r0, r8
 80004c8:	e791      	b.n	80003ee <__udivmoddi4+0x1e6>
 80004ca:	4681      	mov	r9, r0
 80004cc:	e7be      	b.n	800044c <__udivmoddi4+0x244>
 80004ce:	4601      	mov	r1, r0
 80004d0:	e778      	b.n	80003c4 <__udivmoddi4+0x1bc>
 80004d2:	3802      	subs	r0, #2
 80004d4:	443c      	add	r4, r7
 80004d6:	e745      	b.n	8000364 <__udivmoddi4+0x15c>
 80004d8:	4608      	mov	r0, r1
 80004da:	e708      	b.n	80002ee <__udivmoddi4+0xe6>
 80004dc:	f1a8 0802 	sub.w	r8, r8, #2
 80004e0:	443d      	add	r5, r7
 80004e2:	e72b      	b.n	800033c <__udivmoddi4+0x134>

080004e4 <__aeabi_idiv0>:
 80004e4:	4770      	bx	lr
 80004e6:	bf00      	nop

080004e8 <HAL_InitTick>:
  *       implementation  in user file.
  * @param TickPriority Tick interrupt priority.
  * @retval HAL status
  */
__weak HAL_StatusTypeDef HAL_InitTick(uint32_t TickPriority)
{
 80004e8:	b538      	push	{r3, r4, r5, lr}
  /* Configure the SysTick to have interrupt in 1ms time basis*/
  if (HAL_SYSTICK_Config(SystemCoreClock / (1000U / uwTickFreq)) > 0U)
 80004ea:	4a0e      	ldr	r2, [pc, #56]	; (8000524 <HAL_InitTick+0x3c>)
 80004ec:	4b0e      	ldr	r3, [pc, #56]	; (8000528 <HAL_InitTick+0x40>)
{
 80004ee:	4605      	mov	r5, r0
  if (HAL_SYSTICK_Config(SystemCoreClock / (1000U / uwTickFreq)) > 0U)
 80004f0:	7818      	ldrb	r0, [r3, #0]
 80004f2:	f44f 737a 	mov.w	r3, #1000	; 0x3e8
 80004f6:	fbb3 f3f0 	udiv	r3, r3, r0
 80004fa:	6810      	ldr	r0, [r2, #0]
 80004fc:	fbb0 f0f3 	udiv	r0, r0, r3
 8000500:	f000 f89c 	bl	800063c <HAL_SYSTICK_Config>
 8000504:	4604      	mov	r4, r0
 8000506:	b958      	cbnz	r0, 8000520 <HAL_InitTick+0x38>
  {
    return HAL_ERROR;
  }

  /* Configure the SysTick IRQ priority */
  if (TickPriority < (1UL << __NVIC_PRIO_BITS))
 8000508:	2d0f      	cmp	r5, #15
 800050a:	d809      	bhi.n	8000520 <HAL_InitTick+0x38>
  {
    HAL_NVIC_SetPriority(SysTick_IRQn, TickPriority, 0U);
 800050c:	4602      	mov	r2, r0
 800050e:	4629      	mov	r1, r5
 8000510:	f04f 30ff 	mov.w	r0, #4294967295
 8000514:	f000 f85e 	bl	80005d4 <HAL_NVIC_SetPriority>
    uwTickPrio = TickPriority;
 8000518:	4b04      	ldr	r3, [pc, #16]	; (800052c <HAL_InitTick+0x44>)
 800051a:	4620      	mov	r0, r4
 800051c:	601d      	str	r5, [r3, #0]
 800051e:	bd38      	pop	{r3, r4, r5, pc}
    return HAL_ERROR;
 8000520:	2001      	movs	r0, #1
    return HAL_ERROR;
  }

  /* Return function status */
  return HAL_OK;
}
 8000522:	bd38      	pop	{r3, r4, r5, pc}
 8000524:	20000008 	.word	0x20000008
 8000528:	20000000 	.word	0x20000000
 800052c:	20000004 	.word	0x20000004

08000530 <HAL_Init>:
{
 8000530:	b508      	push	{r3, lr}
  __HAL_FLASH_INSTRUCTION_CACHE_ENABLE();
 8000532:	4b0b      	ldr	r3, [pc, #44]	; (8000560 <HAL_Init+0x30>)
 8000534:	681a      	ldr	r2, [r3, #0]
 8000536:	f442 7200 	orr.w	r2, r2, #512	; 0x200
 800053a:	601a      	str	r2, [r3, #0]
  __HAL_FLASH_DATA_CACHE_ENABLE();
 800053c:	681a      	ldr	r2, [r3, #0]
 800053e:	f442 6280 	orr.w	r2, r2, #1024	; 0x400
 8000542:	601a      	str	r2, [r3, #0]
  __HAL_FLASH_PREFETCH_BUFFER_ENABLE();
 8000544:	681a      	ldr	r2, [r3, #0]
 8000546:	f442 7280 	orr.w	r2, r2, #256	; 0x100
 800054a:	601a      	str	r2, [r3, #0]
  HAL_NVIC_SetPriorityGrouping(NVIC_PRIORITYGROUP_4);
 800054c:	2003      	movs	r0, #3
 800054e:	f000 f82f 	bl	80005b0 <HAL_NVIC_SetPriorityGrouping>
  HAL_InitTick(TICK_INT_PRIORITY);
 8000552:	2000      	movs	r0, #0
 8000554:	f7ff ffc8 	bl	80004e8 <HAL_InitTick>
  HAL_MspInit();
 8000558:	f000 fdd6 	bl	8001108 <HAL_MspInit>
}
 800055c:	2000      	movs	r0, #0
 800055e:	bd08      	pop	{r3, pc}
 8000560:	40023c00 	.word	0x40023c00

08000564 <HAL_IncTick>:
  *      implementations in user file.
  * @retval None
  */
__weak void HAL_IncTick(void)
{
  uwTick += uwTickFreq;
 8000564:	4a03      	ldr	r2, [pc, #12]	; (8000574 <HAL_IncTick+0x10>)
 8000566:	4b04      	ldr	r3, [pc, #16]	; (8000578 <HAL_IncTick+0x14>)
 8000568:	6811      	ldr	r1, [r2, #0]
 800056a:	781b      	ldrb	r3, [r3, #0]
 800056c:	440b      	add	r3, r1
 800056e:	6013      	str	r3, [r2, #0]
 8000570:	4770      	bx	lr
 8000572:	bf00      	nop
 8000574:	20000028 	.word	0x20000028
 8000578:	20000000 	.word	0x20000000

0800057c <HAL_GetTick>:
  *       implementations in user file.
  * @retval tick value
  */
__weak uint32_t HAL_GetTick(void)
{
  return uwTick;
 800057c:	4b01      	ldr	r3, [pc, #4]	; (8000584 <HAL_GetTick+0x8>)
 800057e:	6818      	ldr	r0, [r3, #0]
}
 8000580:	4770      	bx	lr
 8000582:	bf00      	nop
 8000584:	20000028 	.word	0x20000028

08000588 <HAL_Delay>:
  *       implementations in user file.
  * @param Delay specifies the delay time length, in milliseconds.
  * @retval None
  */
__weak void HAL_Delay(uint32_t Delay)
{
 8000588:	b538      	push	{r3, r4, r5, lr}
 800058a:	4604      	mov	r4, r0
  uint32_t tickstart = HAL_GetTick();
 800058c:	f7ff fff6 	bl	800057c <HAL_GetTick>
  uint32_t wait = Delay;

  /* Add a freq to guarantee minimum wait */
  if (wait < HAL_MAX_DELAY)
 8000590:	1c63      	adds	r3, r4, #1
  {
    wait += (uint32_t)(uwTickFreq);
 8000592:	bf1c      	itt	ne
 8000594:	4b05      	ldrne	r3, [pc, #20]	; (80005ac <HAL_Delay+0x24>)
 8000596:	781b      	ldrbne	r3, [r3, #0]
  uint32_t tickstart = HAL_GetTick();
 8000598:	4605      	mov	r5, r0
    wait += (uint32_t)(uwTickFreq);
 800059a:	bf18      	it	ne
 800059c:	18e4      	addne	r4, r4, r3
  }

  while((HAL_GetTick() - tickstart) < wait)
 800059e:	f7ff ffed 	bl	800057c <HAL_GetTick>
 80005a2:	1b40      	subs	r0, r0, r5
 80005a4:	4284      	cmp	r4, r0
 80005a6:	d8fa      	bhi.n	800059e <HAL_Delay+0x16>
  {
  }
}
 80005a8:	bd38      	pop	{r3, r4, r5, pc}
 80005aa:	bf00      	nop
 80005ac:	20000000 	.word	0x20000000

080005b0 <HAL_NVIC_SetPriorityGrouping>:
__STATIC_INLINE void __NVIC_SetPriorityGrouping(uint32_t PriorityGroup)
{
  uint32_t reg_value;
  uint32_t PriorityGroupTmp = (PriorityGroup & (uint32_t)0x07UL);             /* only values 0..7 are used          */

  reg_value  =  SCB->AIRCR;                                                   /* read old register configuration    */
 80005b0:	4a07      	ldr	r2, [pc, #28]	; (80005d0 <HAL_NVIC_SetPriorityGrouping+0x20>)
 80005b2:	68d3      	ldr	r3, [r2, #12]
  reg_value &= ~((uint32_t)(SCB_AIRCR_VECTKEY_Msk | SCB_AIRCR_PRIGROUP_Msk)); /* clear bits to change               */
 80005b4:	f423 63e0 	bic.w	r3, r3, #1792	; 0x700
 80005b8:	041b      	lsls	r3, r3, #16
 80005ba:	0c1b      	lsrs	r3, r3, #16
 80005bc:	f043 63bf 	orr.w	r3, r3, #100139008	; 0x5f80000
  reg_value  =  (reg_value                                   |
                ((uint32_t)0x5FAUL << SCB_AIRCR_VECTKEY_Pos) |
                (PriorityGroupTmp << SCB_AIRCR_PRIGROUP_Pos)  );              /* Insert write key and priority group */
 80005c0:	0200      	lsls	r0, r0, #8
 80005c2:	f443 3300 	orr.w	r3, r3, #131072	; 0x20000
 80005c6:	f400 60e0 	and.w	r0, r0, #1792	; 0x700
  reg_value  =  (reg_value                                   |
 80005ca:	4303      	orrs	r3, r0
  SCB->AIRCR =  reg_value;
 80005cc:	60d3      	str	r3, [r2, #12]
 80005ce:	4770      	bx	lr
 80005d0:	e000ed00 	.word	0xe000ed00

080005d4 <HAL_NVIC_SetPriority>:
  \details Reads the priority grouping field from the NVIC Interrupt Controller.
  \return                Priority grouping field (SCB->AIRCR [10:8] PRIGROUP field).
 */
__STATIC_INLINE uint32_t __NVIC_GetPriorityGrouping(void)
{
  return ((uint32_t)((SCB->AIRCR & SCB_AIRCR_PRIGROUP_Msk) >> SCB_AIRCR_PRIGROUP_Pos));
 80005d4:	4b17      	ldr	r3, [pc, #92]	; (8000634 <HAL_NVIC_SetPriority+0x60>)
  *         This parameter can be a value between 0 and 15
  *         A lower priority value indicates a higher priority.          
  * @retval None
  */
void HAL_NVIC_SetPriority(IRQn_Type IRQn, uint32_t PreemptPriority, uint32_t SubPriority)
{ 
 80005d6:	b530      	push	{r4, r5, lr}
 80005d8:	68dc      	ldr	r4, [r3, #12]
 80005da:	f3c4 2402 	ubfx	r4, r4, #8, #3
{
  uint32_t PriorityGroupTmp = (PriorityGroup & (uint32_t)0x07UL);   /* only values 0..7 are used          */
  uint32_t PreemptPriorityBits;
  uint32_t SubPriorityBits;

  PreemptPriorityBits = ((7UL - PriorityGroupTmp) > (uint32_t)(__NVIC_PRIO_BITS)) ? (uint32_t)(__NVIC_PRIO_BITS) : (uint32_t)(7UL - PriorityGroupTmp);
 80005de:	f1c4 0307 	rsb	r3, r4, #7
  SubPriorityBits     = ((PriorityGroupTmp + (uint32_t)(__NVIC_PRIO_BITS)) < (uint32_t)7UL) ? (uint32_t)0UL : (uint32_t)((PriorityGroupTmp - 7UL) + (uint32_t)(__NVIC_PRIO_BITS));
 80005e2:	1d25      	adds	r5, r4, #4
  PreemptPriorityBits = ((7UL - PriorityGroupTmp) > (uint32_t)(__NVIC_PRIO_BITS)) ? (uint32_t)(__NVIC_PRIO_BITS) : (uint32_t)(7UL - PriorityGroupTmp);
 80005e4:	2b04      	cmp	r3, #4
 80005e6:	bf28      	it	cs
 80005e8:	2304      	movcs	r3, #4
  SubPriorityBits     = ((PriorityGroupTmp + (uint32_t)(__NVIC_PRIO_BITS)) < (uint32_t)7UL) ? (uint32_t)0UL : (uint32_t)((PriorityGroupTmp - 7UL) + (uint32_t)(__NVIC_PRIO_BITS));
 80005ea:	2d06      	cmp	r5, #6

  return (
           ((PreemptPriority & (uint32_t)((1UL << (PreemptPriorityBits)) - 1UL)) << SubPriorityBits) |
 80005ec:	f04f 0501 	mov.w	r5, #1
 80005f0:	fa05 f303 	lsl.w	r3, r5, r3
 80005f4:	f103 33ff 	add.w	r3, r3, #4294967295
  SubPriorityBits     = ((PriorityGroupTmp + (uint32_t)(__NVIC_PRIO_BITS)) < (uint32_t)7UL) ? (uint32_t)0UL : (uint32_t)((PriorityGroupTmp - 7UL) + (uint32_t)(__NVIC_PRIO_BITS));
 80005f8:	bf8c      	ite	hi
 80005fa:	3c03      	subhi	r4, #3
 80005fc:	2400      	movls	r4, #0
           ((PreemptPriority & (uint32_t)((1UL << (PreemptPriorityBits)) - 1UL)) << SubPriorityBits) |
 80005fe:	4019      	ands	r1, r3
 8000600:	40a1      	lsls	r1, r4
           ((SubPriority     & (uint32_t)((1UL << (SubPriorityBits    )) - 1UL)))
 8000602:	fa05 f404 	lsl.w	r4, r5, r4
 8000606:	3c01      	subs	r4, #1
 8000608:	4022      	ands	r2, r4
  if ((int32_t)(IRQn) >= 0)
 800060a:	2800      	cmp	r0, #0
           ((PreemptPriority & (uint32_t)((1UL << (PreemptPriorityBits)) - 1UL)) << SubPriorityBits) |
 800060c:	ea42 0201 	orr.w	r2, r2, r1
 8000610:	ea4f 1202 	mov.w	r2, r2, lsl #4
    NVIC->IP[((uint32_t)IRQn)]               = (uint8_t)((priority << (8U - __NVIC_PRIO_BITS)) & (uint32_t)0xFFUL);
 8000614:	bfad      	iteet	ge
 8000616:	f100 4060 	addge.w	r0, r0, #3758096384	; 0xe0000000
    SCB->SHP[(((uint32_t)IRQn) & 0xFUL)-4UL] = (uint8_t)((priority << (8U - __NVIC_PRIO_BITS)) & (uint32_t)0xFFUL);
 800061a:	f000 000f 	andlt.w	r0, r0, #15
 800061e:	4b06      	ldrlt	r3, [pc, #24]	; (8000638 <HAL_NVIC_SetPriority+0x64>)
    NVIC->IP[((uint32_t)IRQn)]               = (uint8_t)((priority << (8U - __NVIC_PRIO_BITS)) & (uint32_t)0xFFUL);
 8000620:	f500 4061 	addge.w	r0, r0, #57600	; 0xe100
    SCB->SHP[(((uint32_t)IRQn) & 0xFUL)-4UL] = (uint8_t)((priority << (8U - __NVIC_PRIO_BITS)) & (uint32_t)0xFFUL);
 8000624:	bfb5      	itete	lt
 8000626:	b2d2      	uxtblt	r2, r2
    NVIC->IP[((uint32_t)IRQn)]               = (uint8_t)((priority << (8U - __NVIC_PRIO_BITS)) & (uint32_t)0xFFUL);
 8000628:	b2d2      	uxtbge	r2, r2
    SCB->SHP[(((uint32_t)IRQn) & 0xFUL)-4UL] = (uint8_t)((priority << (8U - __NVIC_PRIO_BITS)) & (uint32_t)0xFFUL);
 800062a:	541a      	strblt	r2, [r3, r0]
    NVIC->IP[((uint32_t)IRQn)]               = (uint8_t)((priority << (8U - __NVIC_PRIO_BITS)) & (uint32_t)0xFFUL);
 800062c:	f880 2300 	strbge.w	r2, [r0, #768]	; 0x300
 8000630:	bd30      	pop	{r4, r5, pc}
 8000632:	bf00      	nop
 8000634:	e000ed00 	.word	0xe000ed00
 8000638:	e000ed14 	.word	0xe000ed14

0800063c <HAL_SYSTICK_Config>:
           function <b>SysTick_Config</b> is not included. In this case, the file <b><i>device</i>.h</b>
           must contain a vendor-specific implementation of this function.
 */
__STATIC_INLINE uint32_t SysTick_Config(uint32_t ticks)
{
  if ((ticks - 1UL) > SysTick_LOAD_RELOAD_Msk)
 800063c:	3801      	subs	r0, #1
 800063e:	f1b0 7f80 	cmp.w	r0, #16777216	; 0x1000000
 8000642:	d20a      	bcs.n	800065a <HAL_SYSTICK_Config+0x1e>
  {
    return (1UL);                                                   /* Reload value impossible */
  }

  SysTick->LOAD  = (uint32_t)(ticks - 1UL);                         /* set reload register */
 8000644:	4b06      	ldr	r3, [pc, #24]	; (8000660 <HAL_SYSTICK_Config+0x24>)
    SCB->SHP[(((uint32_t)IRQn) & 0xFUL)-4UL] = (uint8_t)((priority << (8U - __NVIC_PRIO_BITS)) & (uint32_t)0xFFUL);
 8000646:	4a07      	ldr	r2, [pc, #28]	; (8000664 <HAL_SYSTICK_Config+0x28>)
  SysTick->LOAD  = (uint32_t)(ticks - 1UL);                         /* set reload register */
 8000648:	6058      	str	r0, [r3, #4]
    SCB->SHP[(((uint32_t)IRQn) & 0xFUL)-4UL] = (uint8_t)((priority << (8U - __NVIC_PRIO_BITS)) & (uint32_t)0xFFUL);
 800064a:	21f0      	movs	r1, #240	; 0xf0
 800064c:	f882 1023 	strb.w	r1, [r2, #35]	; 0x23
  NVIC_SetPriority (SysTick_IRQn, (1UL << __NVIC_PRIO_BITS) - 1UL); /* set Priority for Systick Interrupt */
  SysTick->VAL   = 0UL;                                             /* Load the SysTick Counter Value */
 8000650:	2000      	movs	r0, #0
  SysTick->CTRL  = SysTick_CTRL_CLKSOURCE_Msk |
 8000652:	2207      	movs	r2, #7
  SysTick->VAL   = 0UL;                                             /* Load the SysTick Counter Value */
 8000654:	6098      	str	r0, [r3, #8]
  SysTick->CTRL  = SysTick_CTRL_CLKSOURCE_Msk |
 8000656:	601a      	str	r2, [r3, #0]
 8000658:	4770      	bx	lr
    return (1UL);                                                   /* Reload value impossible */
 800065a:	2001      	movs	r0, #1
  *                  - 1  Function failed.
  */
uint32_t HAL_SYSTICK_Config(uint32_t TicksNumb)
{
   return SysTick_Config(TicksNumb);
}
 800065c:	4770      	bx	lr
 800065e:	bf00      	nop
 8000660:	e000e010 	.word	0xe000e010
 8000664:	e000ed00 	.word	0xe000ed00

08000668 <HAL_GPIO_Init>:
  * @param  GPIO_Init pointer to a GPIO_InitTypeDef structure that contains
  *         the configuration information for the specified GPIO peripheral.
  * @retval None
  */
void HAL_GPIO_Init(GPIO_TypeDef  *GPIOx, GPIO_InitTypeDef *GPIO_Init)
{
 8000668:	e92d 4ff0 	stmdb	sp!, {r4, r5, r6, r7, r8, r9, sl, fp, lr}
 800066c:	b085      	sub	sp, #20
  for(position = 0U; position < GPIO_NUMBER; position++)
  {
    /* Get the IO position */
    ioposition = 0x01U << position;
    /* Get the current IO position */
    iocurrent = (uint32_t)(GPIO_Init->Pin) & ioposition;
 800066e:	680b      	ldr	r3, [r1, #0]
      /*--------------------- EXTI Mode Configuration ------------------------*/
      /* Configure the External Interrupt or event for the current IO */
      if((GPIO_Init->Mode & EXTI_MODE) == EXTI_MODE)
      {
        /* Enable SYSCFG Clock */
        __HAL_RCC_SYSCFG_CLK_ENABLE();
 8000670:	f8df 819c 	ldr.w	r8, [pc, #412]	; 8000810 <HAL_GPIO_Init+0x1a8>
        temp &= ~(0x0FU << (4U * (position & 0x03U)));
        temp |= ((uint32_t)(GPIO_GET_INDEX(GPIOx)) << (4U * (position & 0x03U)));
        SYSCFG->EXTICR[position >> 2U] = temp;

        /* Clear EXTI line configuration */
        temp = EXTI->IMR;
 8000674:	4a64      	ldr	r2, [pc, #400]	; (8000808 <HAL_GPIO_Init+0x1a0>)
    iocurrent = (uint32_t)(GPIO_Init->Pin) & ioposition;
 8000676:	9301      	str	r3, [sp, #4]
    ioposition = 0x01U << position;
 8000678:	f04f 0901 	mov.w	r9, #1
  for(position = 0U; position < GPIO_NUMBER; position++)
 800067c:	2300      	movs	r3, #0
    iocurrent = (uint32_t)(GPIO_Init->Pin) & ioposition;
 800067e:	9c01      	ldr	r4, [sp, #4]
    ioposition = 0x01U << position;
 8000680:	fa09 f703 	lsl.w	r7, r9, r3
    iocurrent = (uint32_t)(GPIO_Init->Pin) & ioposition;
 8000684:	ea07 0604 	and.w	r6, r7, r4
    if(iocurrent == ioposition)
 8000688:	42b7      	cmp	r7, r6
 800068a:	f040 80ad 	bne.w	80007e8 <HAL_GPIO_Init+0x180>
      if((GPIO_Init->Mode == GPIO_MODE_AF_PP) || (GPIO_Init->Mode == GPIO_MODE_AF_OD))
 800068e:	684c      	ldr	r4, [r1, #4]
 8000690:	f024 0a10 	bic.w	sl, r4, #16
 8000694:	f1ba 0f02 	cmp.w	sl, #2
 8000698:	d116      	bne.n	80006c8 <HAL_GPIO_Init+0x60>
        temp = GPIOx->AFR[position >> 3U];
 800069a:	ea4f 0cd3 	mov.w	ip, r3, lsr #3
 800069e:	eb00 0c8c 	add.w	ip, r0, ip, lsl #2
        temp &= ~(0xFU << ((uint32_t)(position & 0x07U) * 4U)) ;
 80006a2:	f003 0b07 	and.w	fp, r3, #7
        temp = GPIOx->AFR[position >> 3U];
 80006a6:	f8dc 5020 	ldr.w	r5, [ip, #32]
        temp &= ~(0xFU << ((uint32_t)(position & 0x07U) * 4U)) ;
 80006aa:	ea4f 0b8b 	mov.w	fp, fp, lsl #2
 80006ae:	f04f 0e0f 	mov.w	lr, #15
 80006b2:	fa0e fe0b 	lsl.w	lr, lr, fp
 80006b6:	ea25 0e0e 	bic.w	lr, r5, lr
        temp |= ((uint32_t)(GPIO_Init->Alternate) << (((uint32_t)position & 0x07U) * 4U));
 80006ba:	690d      	ldr	r5, [r1, #16]
 80006bc:	fa05 f50b 	lsl.w	r5, r5, fp
 80006c0:	ea45 050e 	orr.w	r5, r5, lr
        GPIOx->AFR[position >> 3U] = temp;
 80006c4:	f8cc 5020 	str.w	r5, [ip, #32]
 80006c8:	ea4f 0c43 	mov.w	ip, r3, lsl #1
      temp &= ~(GPIO_MODER_MODER0 << (position * 2U));
 80006cc:	2503      	movs	r5, #3
      temp = GPIOx->MODER;
 80006ce:	f8d0 b000 	ldr.w	fp, [r0]
      temp &= ~(GPIO_MODER_MODER0 << (position * 2U));
 80006d2:	fa05 f50c 	lsl.w	r5, r5, ip
 80006d6:	43ed      	mvns	r5, r5
      temp |= ((GPIO_Init->Mode & GPIO_MODE) << (position * 2U));
 80006d8:	f004 0e03 	and.w	lr, r4, #3
      temp &= ~(GPIO_MODER_MODER0 << (position * 2U));
 80006dc:	ea0b 0b05 	and.w	fp, fp, r5
      temp |= ((GPIO_Init->Mode & GPIO_MODE) << (position * 2U));
 80006e0:	fa0e fe0c 	lsl.w	lr, lr, ip
      if((GPIO_Init->Mode == GPIO_MODE_OUTPUT_PP) || (GPIO_Init->Mode == GPIO_MODE_AF_PP) ||
 80006e4:	f10a 3aff 	add.w	sl, sl, #4294967295
      temp |= ((GPIO_Init->Mode & GPIO_MODE) << (position * 2U));
 80006e8:	ea4e 0e0b 	orr.w	lr, lr, fp
      if((GPIO_Init->Mode == GPIO_MODE_OUTPUT_PP) || (GPIO_Init->Mode == GPIO_MODE_AF_PP) ||
 80006ec:	f1ba 0f01 	cmp.w	sl, #1
      temp &= ~(GPIO_MODER_MODER0 << (position * 2U));
 80006f0:	9500      	str	r5, [sp, #0]
      GPIOx->MODER = temp;
 80006f2:	f8c0 e000 	str.w	lr, [r0]
      if((GPIO_Init->Mode == GPIO_MODE_OUTPUT_PP) || (GPIO_Init->Mode == GPIO_MODE_AF_PP) ||
 80006f6:	d815      	bhi.n	8000724 <HAL_GPIO_Init+0xbc>
        temp = GPIOx->OSPEEDR; 
 80006f8:	f8d0 e008 	ldr.w	lr, [r0, #8]
        temp &= ~(GPIO_OSPEEDER_OSPEEDR0 << (position * 2U));
 80006fc:	ea05 0e0e 	and.w	lr, r5, lr
        temp |= (GPIO_Init->Speed << (position * 2U));
 8000700:	68cd      	ldr	r5, [r1, #12]
 8000702:	fa05 fa0c 	lsl.w	sl, r5, ip
 8000706:	ea4a 0e0e 	orr.w	lr, sl, lr
        GPIOx->OSPEEDR = temp;
 800070a:	f8c0 e008 	str.w	lr, [r0, #8]
        temp = GPIOx->OTYPER;
 800070e:	f8d0 e004 	ldr.w	lr, [r0, #4]
        temp &= ~(GPIO_OTYPER_OT_0 << position) ;
 8000712:	ea2e 0707 	bic.w	r7, lr, r7
        temp |= (((GPIO_Init->Mode & GPIO_OUTPUT_TYPE) >> 4U) << position);
 8000716:	f3c4 1e00 	ubfx	lr, r4, #4, #1
 800071a:	fa0e fe03 	lsl.w	lr, lr, r3
 800071e:	ea4e 0707 	orr.w	r7, lr, r7
        GPIOx->OTYPER = temp;
 8000722:	6047      	str	r7, [r0, #4]
      temp = GPIOx->PUPDR;
 8000724:	68c7      	ldr	r7, [r0, #12]
      temp &= ~(GPIO_PUPDR_PUPDR0 << (position * 2U));
 8000726:	9d00      	ldr	r5, [sp, #0]
 8000728:	403d      	ands	r5, r7
      temp |= ((GPIO_Init->Pull) << (position * 2U));
 800072a:	688f      	ldr	r7, [r1, #8]
 800072c:	fa07 f70c 	lsl.w	r7, r7, ip
 8000730:	433d      	orrs	r5, r7
      GPIOx->PUPDR = temp;
 8000732:	60c5      	str	r5, [r0, #12]
      if((GPIO_Init->Mode & EXTI_MODE) == EXTI_MODE)
 8000734:	00e5      	lsls	r5, r4, #3
 8000736:	d557      	bpl.n	80007e8 <HAL_GPIO_Init+0x180>
        __HAL_RCC_SYSCFG_CLK_ENABLE();
 8000738:	f04f 0b00 	mov.w	fp, #0
 800073c:	f8cd b00c 	str.w	fp, [sp, #12]
 8000740:	f8d8 7044 	ldr.w	r7, [r8, #68]	; 0x44
        temp |= ((uint32_t)(GPIO_GET_INDEX(GPIOx)) << (4U * (position & 0x03U)));
 8000744:	4d31      	ldr	r5, [pc, #196]	; (800080c <HAL_GPIO_Init+0x1a4>)
        __HAL_RCC_SYSCFG_CLK_ENABLE();
 8000746:	f447 4780 	orr.w	r7, r7, #16384	; 0x4000
 800074a:	f8c8 7044 	str.w	r7, [r8, #68]	; 0x44
 800074e:	f8d8 7044 	ldr.w	r7, [r8, #68]	; 0x44
 8000752:	f407 4780 	and.w	r7, r7, #16384	; 0x4000
 8000756:	9703      	str	r7, [sp, #12]
 8000758:	9f03      	ldr	r7, [sp, #12]
 800075a:	f023 0703 	bic.w	r7, r3, #3
 800075e:	f107 4780 	add.w	r7, r7, #1073741824	; 0x40000000
 8000762:	f507 379c 	add.w	r7, r7, #79872	; 0x13800
        temp &= ~(0x0FU << (4U * (position & 0x03U)));
 8000766:	f003 0c03 	and.w	ip, r3, #3
        temp = SYSCFG->EXTICR[position >> 2U];
 800076a:	f8d7 a008 	ldr.w	sl, [r7, #8]
        temp &= ~(0x0FU << (4U * (position & 0x03U)));
 800076e:	ea4f 0c8c 	mov.w	ip, ip, lsl #2
 8000772:	f04f 0e0f 	mov.w	lr, #15
 8000776:	fa0e fe0c 	lsl.w	lr, lr, ip
        temp |= ((uint32_t)(GPIO_GET_INDEX(GPIOx)) << (4U * (position & 0x03U)));
 800077a:	42a8      	cmp	r0, r5
        temp &= ~(0x0FU << (4U * (position & 0x03U)));
 800077c:	ea2a 0e0e 	bic.w	lr, sl, lr
        temp |= ((uint32_t)(GPIO_GET_INDEX(GPIOx)) << (4U * (position & 0x03U)));
 8000780:	d039      	beq.n	80007f6 <HAL_GPIO_Init+0x18e>
 8000782:	f505 6580 	add.w	r5, r5, #1024	; 0x400
 8000786:	42a8      	cmp	r0, r5
 8000788:	d037      	beq.n	80007fa <HAL_GPIO_Init+0x192>
 800078a:	f505 6580 	add.w	r5, r5, #1024	; 0x400
 800078e:	42a8      	cmp	r0, r5
 8000790:	d035      	beq.n	80007fe <HAL_GPIO_Init+0x196>
 8000792:	f505 6580 	add.w	r5, r5, #1024	; 0x400
 8000796:	42a8      	cmp	r0, r5
 8000798:	d033      	beq.n	8000802 <HAL_GPIO_Init+0x19a>
 800079a:	f505 6580 	add.w	r5, r5, #1024	; 0x400
 800079e:	42a8      	cmp	r0, r5
 80007a0:	bf14      	ite	ne
 80007a2:	2507      	movne	r5, #7
 80007a4:	2504      	moveq	r5, #4
 80007a6:	fa05 f50c 	lsl.w	r5, r5, ip
 80007aa:	ea45 050e 	orr.w	r5, r5, lr
        SYSCFG->EXTICR[position >> 2U] = temp;
 80007ae:	60bd      	str	r5, [r7, #8]
        temp = EXTI->IMR;
 80007b0:	6815      	ldr	r5, [r2, #0]
        temp &= ~((uint32_t)iocurrent);
 80007b2:	43f7      	mvns	r7, r6
        if((GPIO_Init->Mode & GPIO_MODE_IT) == GPIO_MODE_IT)
 80007b4:	f414 3f80 	tst.w	r4, #65536	; 0x10000
        temp &= ~((uint32_t)iocurrent);
 80007b8:	bf0c      	ite	eq
 80007ba:	403d      	andeq	r5, r7
        {
          temp |= iocurrent;
 80007bc:	4335      	orrne	r5, r6
        }
        EXTI->IMR = temp;
 80007be:	6015      	str	r5, [r2, #0]

        temp = EXTI->EMR;
 80007c0:	6855      	ldr	r5, [r2, #4]
        temp &= ~((uint32_t)iocurrent);
        if((GPIO_Init->Mode & GPIO_MODE_EVT) == GPIO_MODE_EVT)
 80007c2:	f414 3f00 	tst.w	r4, #131072	; 0x20000
        temp &= ~((uint32_t)iocurrent);
 80007c6:	bf0c      	ite	eq
 80007c8:	403d      	andeq	r5, r7
        {
          temp |= iocurrent;
 80007ca:	4335      	orrne	r5, r6
        }
        EXTI->EMR = temp;
 80007cc:	6055      	str	r5, [r2, #4]

        /* Clear Rising Falling edge configuration */
        temp = EXTI->RTSR;
 80007ce:	6895      	ldr	r5, [r2, #8]
        temp &= ~((uint32_t)iocurrent);
        if((GPIO_Init->Mode & RISING_EDGE) == RISING_EDGE)
 80007d0:	f414 1f80 	tst.w	r4, #1048576	; 0x100000
        temp &= ~((uint32_t)iocurrent);
 80007d4:	bf0c      	ite	eq
 80007d6:	403d      	andeq	r5, r7
        {
          temp |= iocurrent;
 80007d8:	4335      	orrne	r5, r6
        }
        EXTI->RTSR = temp;
 80007da:	6095      	str	r5, [r2, #8]

        temp = EXTI->FTSR;
 80007dc:	68d5      	ldr	r5, [r2, #12]
        temp &= ~((uint32_t)iocurrent);
        if((GPIO_Init->Mode & FALLING_EDGE) == FALLING_EDGE)
 80007de:	02a4      	lsls	r4, r4, #10
        temp &= ~((uint32_t)iocurrent);
 80007e0:	bf54      	ite	pl
 80007e2:	403d      	andpl	r5, r7
        {
          temp |= iocurrent;
 80007e4:	4335      	orrmi	r5, r6
        }
        EXTI->FTSR = temp;
 80007e6:	60d5      	str	r5, [r2, #12]
  for(position = 0U; position < GPIO_NUMBER; position++)
 80007e8:	3301      	adds	r3, #1
 80007ea:	2b10      	cmp	r3, #16
 80007ec:	f47f af47 	bne.w	800067e <HAL_GPIO_Init+0x16>
      }
    }
  }
}
 80007f0:	b005      	add	sp, #20
 80007f2:	e8bd 8ff0 	ldmia.w	sp!, {r4, r5, r6, r7, r8, r9, sl, fp, pc}
        temp |= ((uint32_t)(GPIO_GET_INDEX(GPIOx)) << (4U * (position & 0x03U)));
 80007f6:	465d      	mov	r5, fp
 80007f8:	e7d5      	b.n	80007a6 <HAL_GPIO_Init+0x13e>
 80007fa:	2501      	movs	r5, #1
 80007fc:	e7d3      	b.n	80007a6 <HAL_GPIO_Init+0x13e>
 80007fe:	2502      	movs	r5, #2
 8000800:	e7d1      	b.n	80007a6 <HAL_GPIO_Init+0x13e>
 8000802:	2503      	movs	r5, #3
 8000804:	e7cf      	b.n	80007a6 <HAL_GPIO_Init+0x13e>
 8000806:	bf00      	nop
 8000808:	40013c00 	.word	0x40013c00
 800080c:	40020000 	.word	0x40020000
 8000810:	40023800 	.word	0x40023800

08000814 <HAL_GPIO_WritePin>:
{
  /* Check the parameters */
  assert_param(IS_GPIO_PIN(GPIO_Pin));
  assert_param(IS_GPIO_PIN_ACTION(PinState));

  if(PinState != GPIO_PIN_RESET)
 8000814:	b10a      	cbz	r2, 800081a <HAL_GPIO_WritePin+0x6>
  {
    GPIOx->BSRR = GPIO_Pin;
  }
  else
  {
    GPIOx->BSRR = (uint32_t)GPIO_Pin << 16U;
 8000816:	6181      	str	r1, [r0, #24]
 8000818:	4770      	bx	lr
 800081a:	0409      	lsls	r1, r1, #16
 800081c:	e7fb      	b.n	8000816 <HAL_GPIO_WritePin+0x2>

0800081e <HAL_GPIO_TogglePin>:
void HAL_GPIO_TogglePin(GPIO_TypeDef* GPIOx, uint16_t GPIO_Pin)
{
  /* Check the parameters */
  assert_param(IS_GPIO_PIN(GPIO_Pin));

  if ((GPIOx->ODR & GPIO_Pin) == GPIO_Pin)
 800081e:	6943      	ldr	r3, [r0, #20]
 8000820:	ea31 0303 	bics.w	r3, r1, r3
  {
    GPIOx->BSRR = (uint32_t)GPIO_Pin << GPIO_NUMBER;
 8000824:	bf08      	it	eq
 8000826:	0409      	lsleq	r1, r1, #16
  }
  else
  {
    GPIOx->BSRR = GPIO_Pin;
 8000828:	6181      	str	r1, [r0, #24]
 800082a:	4770      	bx	lr

0800082c <HAL_RCC_OscConfig>:
  *         supported by this API. User should request a transition to HSE Off
  *         first and then HSE On or HSE Bypass.
  * @retval HAL status
  */
__weak HAL_StatusTypeDef HAL_RCC_OscConfig(RCC_OscInitTypeDef  *RCC_OscInitStruct)
{
 800082c:	e92d 41f3 	stmdb	sp!, {r0, r1, r4, r5, r6, r7, r8, lr}
  uint32_t tickstart;

  /* Check Null pointer */
  if(RCC_OscInitStruct == NULL)
 8000830:	4604      	mov	r4, r0
 8000832:	b918      	cbnz	r0, 800083c <HAL_RCC_OscConfig+0x10>
  {
    return HAL_ERROR;
 8000834:	2001      	movs	r0, #1
    {
      return HAL_ERROR;
    }
  }
  return HAL_OK;
}
 8000836:	b002      	add	sp, #8
 8000838:	e8bd 81f0 	ldmia.w	sp!, {r4, r5, r6, r7, r8, pc}
  if(((RCC_OscInitStruct->OscillatorType) & RCC_OSCILLATORTYPE_HSE) == RCC_OSCILLATORTYPE_HSE)
 800083c:	6803      	ldr	r3, [r0, #0]
 800083e:	07dd      	lsls	r5, r3, #31
 8000840:	d410      	bmi.n	8000864 <HAL_RCC_OscConfig+0x38>
  if(((RCC_OscInitStruct->OscillatorType) & RCC_OSCILLATORTYPE_HSI) == RCC_OSCILLATORTYPE_HSI)
 8000842:	6823      	ldr	r3, [r4, #0]
 8000844:	0798      	lsls	r0, r3, #30
 8000846:	d458      	bmi.n	80008fa <HAL_RCC_OscConfig+0xce>
  if(((RCC_OscInitStruct->OscillatorType) & RCC_OSCILLATORTYPE_LSI) == RCC_OSCILLATORTYPE_LSI)
 8000848:	6823      	ldr	r3, [r4, #0]
 800084a:	071a      	lsls	r2, r3, #28
 800084c:	f100 809a 	bmi.w	8000984 <HAL_RCC_OscConfig+0x158>
  if(((RCC_OscInitStruct->OscillatorType) & RCC_OSCILLATORTYPE_LSE) == RCC_OSCILLATORTYPE_LSE)
 8000850:	6823      	ldr	r3, [r4, #0]
 8000852:	075b      	lsls	r3, r3, #29
 8000854:	f100 80b8 	bmi.w	80009c8 <HAL_RCC_OscConfig+0x19c>
  if ((RCC_OscInitStruct->PLL.PLLState) != RCC_PLL_NONE)
 8000858:	69a2      	ldr	r2, [r4, #24]
 800085a:	2a00      	cmp	r2, #0
 800085c:	f040 8119 	bne.w	8000a92 <HAL_RCC_OscConfig+0x266>
  return HAL_OK;
 8000860:	2000      	movs	r0, #0
 8000862:	e7e8      	b.n	8000836 <HAL_RCC_OscConfig+0xa>
    if((__HAL_RCC_GET_SYSCLK_SOURCE() == RCC_CFGR_SWS_HSE) ||\
 8000864:	4ba6      	ldr	r3, [pc, #664]	; (8000b00 <HAL_RCC_OscConfig+0x2d4>)
 8000866:	689a      	ldr	r2, [r3, #8]
 8000868:	f002 020c 	and.w	r2, r2, #12
 800086c:	2a04      	cmp	r2, #4
 800086e:	d007      	beq.n	8000880 <HAL_RCC_OscConfig+0x54>
      ((__HAL_RCC_GET_SYSCLK_SOURCE() == RCC_CFGR_SWS_PLL) && ((RCC->PLLCFGR & RCC_PLLCFGR_PLLSRC) == RCC_PLLCFGR_PLLSRC_HSE)))
 8000870:	689a      	ldr	r2, [r3, #8]
 8000872:	f002 020c 	and.w	r2, r2, #12
    if((__HAL_RCC_GET_SYSCLK_SOURCE() == RCC_CFGR_SWS_HSE) ||\
 8000876:	2a08      	cmp	r2, #8
 8000878:	d10a      	bne.n	8000890 <HAL_RCC_OscConfig+0x64>
      ((__HAL_RCC_GET_SYSCLK_SOURCE() == RCC_CFGR_SWS_PLL) && ((RCC->PLLCFGR & RCC_PLLCFGR_PLLSRC) == RCC_PLLCFGR_PLLSRC_HSE)))
 800087a:	685b      	ldr	r3, [r3, #4]
 800087c:	0259      	lsls	r1, r3, #9
 800087e:	d507      	bpl.n	8000890 <HAL_RCC_OscConfig+0x64>
      if((__HAL_RCC_GET_FLAG(RCC_FLAG_HSERDY) != RESET) && (RCC_OscInitStruct->HSEState == RCC_HSE_OFF))
 8000880:	4b9f      	ldr	r3, [pc, #636]	; (8000b00 <HAL_RCC_OscConfig+0x2d4>)
 8000882:	681b      	ldr	r3, [r3, #0]
 8000884:	039a      	lsls	r2, r3, #14
 8000886:	d5dc      	bpl.n	8000842 <HAL_RCC_OscConfig+0x16>
 8000888:	6863      	ldr	r3, [r4, #4]
 800088a:	2b00      	cmp	r3, #0
 800088c:	d1d9      	bne.n	8000842 <HAL_RCC_OscConfig+0x16>
 800088e:	e7d1      	b.n	8000834 <HAL_RCC_OscConfig+0x8>
      __HAL_RCC_HSE_CONFIG(RCC_OscInitStruct->HSEState);
 8000890:	6863      	ldr	r3, [r4, #4]
 8000892:	4d9b      	ldr	r5, [pc, #620]	; (8000b00 <HAL_RCC_OscConfig+0x2d4>)
 8000894:	f5b3 3f80 	cmp.w	r3, #65536	; 0x10000
 8000898:	d111      	bne.n	80008be <HAL_RCC_OscConfig+0x92>
 800089a:	682b      	ldr	r3, [r5, #0]
 800089c:	f443 3380 	orr.w	r3, r3, #65536	; 0x10000
 80008a0:	602b      	str	r3, [r5, #0]
        tickstart = HAL_GetTick();
 80008a2:	f7ff fe6b 	bl	800057c <HAL_GetTick>
        while(__HAL_RCC_GET_FLAG(RCC_FLAG_HSERDY) == RESET)
 80008a6:	4d96      	ldr	r5, [pc, #600]	; (8000b00 <HAL_RCC_OscConfig+0x2d4>)
        tickstart = HAL_GetTick();
 80008a8:	4606      	mov	r6, r0
        while(__HAL_RCC_GET_FLAG(RCC_FLAG_HSERDY) == RESET)
 80008aa:	682b      	ldr	r3, [r5, #0]
 80008ac:	039b      	lsls	r3, r3, #14
 80008ae:	d4c8      	bmi.n	8000842 <HAL_RCC_OscConfig+0x16>
          if((HAL_GetTick() - tickstart ) > HSE_TIMEOUT_VALUE)
 80008b0:	f7ff fe64 	bl	800057c <HAL_GetTick>
 80008b4:	1b80      	subs	r0, r0, r6
 80008b6:	2864      	cmp	r0, #100	; 0x64
 80008b8:	d9f7      	bls.n	80008aa <HAL_RCC_OscConfig+0x7e>
            return HAL_TIMEOUT;
 80008ba:	2003      	movs	r0, #3
 80008bc:	e7bb      	b.n	8000836 <HAL_RCC_OscConfig+0xa>
      __HAL_RCC_HSE_CONFIG(RCC_OscInitStruct->HSEState);
 80008be:	f5b3 2fa0 	cmp.w	r3, #327680	; 0x50000
 80008c2:	d104      	bne.n	80008ce <HAL_RCC_OscConfig+0xa2>
 80008c4:	682b      	ldr	r3, [r5, #0]
 80008c6:	f443 2380 	orr.w	r3, r3, #262144	; 0x40000
 80008ca:	602b      	str	r3, [r5, #0]
 80008cc:	e7e5      	b.n	800089a <HAL_RCC_OscConfig+0x6e>
 80008ce:	682a      	ldr	r2, [r5, #0]
 80008d0:	f422 3280 	bic.w	r2, r2, #65536	; 0x10000
 80008d4:	602a      	str	r2, [r5, #0]
 80008d6:	682a      	ldr	r2, [r5, #0]
 80008d8:	f422 2280 	bic.w	r2, r2, #262144	; 0x40000
 80008dc:	602a      	str	r2, [r5, #0]
      if((RCC_OscInitStruct->HSEState) != RCC_HSE_OFF)
 80008de:	2b00      	cmp	r3, #0
 80008e0:	d1df      	bne.n	80008a2 <HAL_RCC_OscConfig+0x76>
        tickstart = HAL_GetTick();
 80008e2:	f7ff fe4b 	bl	800057c <HAL_GetTick>
 80008e6:	4606      	mov	r6, r0
        while(__HAL_RCC_GET_FLAG(RCC_FLAG_HSERDY) != RESET)
 80008e8:	682b      	ldr	r3, [r5, #0]
 80008ea:	039f      	lsls	r7, r3, #14
 80008ec:	d5a9      	bpl.n	8000842 <HAL_RCC_OscConfig+0x16>
          if((HAL_GetTick() - tickstart ) > HSE_TIMEOUT_VALUE)
 80008ee:	f7ff fe45 	bl	800057c <HAL_GetTick>
 80008f2:	1b80      	subs	r0, r0, r6
 80008f4:	2864      	cmp	r0, #100	; 0x64
 80008f6:	d9f7      	bls.n	80008e8 <HAL_RCC_OscConfig+0xbc>
 80008f8:	e7df      	b.n	80008ba <HAL_RCC_OscConfig+0x8e>
    if((__HAL_RCC_GET_SYSCLK_SOURCE() == RCC_CFGR_SWS_HSI) ||\
 80008fa:	4b81      	ldr	r3, [pc, #516]	; (8000b00 <HAL_RCC_OscConfig+0x2d4>)
 80008fc:	689a      	ldr	r2, [r3, #8]
 80008fe:	f012 0f0c 	tst.w	r2, #12
 8000902:	d007      	beq.n	8000914 <HAL_RCC_OscConfig+0xe8>
      ((__HAL_RCC_GET_SYSCLK_SOURCE() == RCC_CFGR_SWS_PLL) && ((RCC->PLLCFGR & RCC_PLLCFGR_PLLSRC) == RCC_PLLCFGR_PLLSRC_HSI)))
 8000904:	689a      	ldr	r2, [r3, #8]
 8000906:	f002 020c 	and.w	r2, r2, #12
    if((__HAL_RCC_GET_SYSCLK_SOURCE() == RCC_CFGR_SWS_HSI) ||\
 800090a:	2a08      	cmp	r2, #8
 800090c:	d111      	bne.n	8000932 <HAL_RCC_OscConfig+0x106>
      ((__HAL_RCC_GET_SYSCLK_SOURCE() == RCC_CFGR_SWS_PLL) && ((RCC->PLLCFGR & RCC_PLLCFGR_PLLSRC) == RCC_PLLCFGR_PLLSRC_HSI)))
 800090e:	685b      	ldr	r3, [r3, #4]
 8000910:	025e      	lsls	r6, r3, #9
 8000912:	d40e      	bmi.n	8000932 <HAL_RCC_OscConfig+0x106>
      if((__HAL_RCC_GET_FLAG(RCC_FLAG_HSIRDY) != RESET) && (RCC_OscInitStruct->HSIState != RCC_HSI_ON))
 8000914:	4b7a      	ldr	r3, [pc, #488]	; (8000b00 <HAL_RCC_OscConfig+0x2d4>)
 8000916:	681a      	ldr	r2, [r3, #0]
 8000918:	0795      	lsls	r5, r2, #30
 800091a:	d502      	bpl.n	8000922 <HAL_RCC_OscConfig+0xf6>
 800091c:	68e2      	ldr	r2, [r4, #12]
 800091e:	2a01      	cmp	r2, #1
 8000920:	d188      	bne.n	8000834 <HAL_RCC_OscConfig+0x8>
        __HAL_RCC_HSI_CALIBRATIONVALUE_ADJUST(RCC_OscInitStruct->HSICalibrationValue);
 8000922:	681a      	ldr	r2, [r3, #0]
 8000924:	6921      	ldr	r1, [r4, #16]
 8000926:	f022 02f8 	bic.w	r2, r2, #248	; 0xf8
 800092a:	ea42 02c1 	orr.w	r2, r2, r1, lsl #3
 800092e:	601a      	str	r2, [r3, #0]
      if((__HAL_RCC_GET_FLAG(RCC_FLAG_HSIRDY) != RESET) && (RCC_OscInitStruct->HSIState != RCC_HSI_ON))
 8000930:	e78a      	b.n	8000848 <HAL_RCC_OscConfig+0x1c>
      if((RCC_OscInitStruct->HSIState)!= RCC_HSI_OFF)
 8000932:	68e2      	ldr	r2, [r4, #12]
 8000934:	4b73      	ldr	r3, [pc, #460]	; (8000b04 <HAL_RCC_OscConfig+0x2d8>)
 8000936:	b1b2      	cbz	r2, 8000966 <HAL_RCC_OscConfig+0x13a>
        __HAL_RCC_HSI_ENABLE();
 8000938:	2201      	movs	r2, #1
 800093a:	601a      	str	r2, [r3, #0]
        tickstart = HAL_GetTick();
 800093c:	f7ff fe1e 	bl	800057c <HAL_GetTick>
        while(__HAL_RCC_GET_FLAG(RCC_FLAG_HSIRDY) == RESET)
 8000940:	4d6f      	ldr	r5, [pc, #444]	; (8000b00 <HAL_RCC_OscConfig+0x2d4>)
        tickstart = HAL_GetTick();
 8000942:	4606      	mov	r6, r0
        while(__HAL_RCC_GET_FLAG(RCC_FLAG_HSIRDY) == RESET)
 8000944:	682b      	ldr	r3, [r5, #0]
 8000946:	0798      	lsls	r0, r3, #30
 8000948:	d507      	bpl.n	800095a <HAL_RCC_OscConfig+0x12e>
        __HAL_RCC_HSI_CALIBRATIONVALUE_ADJUST(RCC_OscInitStruct->HSICalibrationValue);
 800094a:	682b      	ldr	r3, [r5, #0]
 800094c:	6922      	ldr	r2, [r4, #16]
 800094e:	f023 03f8 	bic.w	r3, r3, #248	; 0xf8
 8000952:	ea43 03c2 	orr.w	r3, r3, r2, lsl #3
 8000956:	602b      	str	r3, [r5, #0]
 8000958:	e776      	b.n	8000848 <HAL_RCC_OscConfig+0x1c>
          if((HAL_GetTick() - tickstart ) > HSI_TIMEOUT_VALUE)
 800095a:	f7ff fe0f 	bl	800057c <HAL_GetTick>
 800095e:	1b80      	subs	r0, r0, r6
 8000960:	2802      	cmp	r0, #2
 8000962:	d9ef      	bls.n	8000944 <HAL_RCC_OscConfig+0x118>
 8000964:	e7a9      	b.n	80008ba <HAL_RCC_OscConfig+0x8e>
        __HAL_RCC_HSI_DISABLE();
 8000966:	601a      	str	r2, [r3, #0]
        tickstart = HAL_GetTick();
 8000968:	f7ff fe08 	bl	800057c <HAL_GetTick>
        while(__HAL_RCC_GET_FLAG(RCC_FLAG_HSIRDY) != RESET)
 800096c:	4d64      	ldr	r5, [pc, #400]	; (8000b00 <HAL_RCC_OscConfig+0x2d4>)
        tickstart = HAL_GetTick();
 800096e:	4606      	mov	r6, r0
        while(__HAL_RCC_GET_FLAG(RCC_FLAG_HSIRDY) != RESET)
 8000970:	682b      	ldr	r3, [r5, #0]
 8000972:	0799      	lsls	r1, r3, #30
 8000974:	f57f af68 	bpl.w	8000848 <HAL_RCC_OscConfig+0x1c>
          if((HAL_GetTick() - tickstart ) > HSI_TIMEOUT_VALUE)
 8000978:	f7ff fe00 	bl	800057c <HAL_GetTick>
 800097c:	1b80      	subs	r0, r0, r6
 800097e:	2802      	cmp	r0, #2
 8000980:	d9f6      	bls.n	8000970 <HAL_RCC_OscConfig+0x144>
 8000982:	e79a      	b.n	80008ba <HAL_RCC_OscConfig+0x8e>
    if((RCC_OscInitStruct->LSIState)!= RCC_LSI_OFF)
 8000984:	6962      	ldr	r2, [r4, #20]
 8000986:	4b60      	ldr	r3, [pc, #384]	; (8000b08 <HAL_RCC_OscConfig+0x2dc>)
 8000988:	b17a      	cbz	r2, 80009aa <HAL_RCC_OscConfig+0x17e>
      __HAL_RCC_LSI_ENABLE();
 800098a:	2201      	movs	r2, #1
 800098c:	601a      	str	r2, [r3, #0]
      tickstart = HAL_GetTick();
 800098e:	f7ff fdf5 	bl	800057c <HAL_GetTick>
      while(__HAL_RCC_GET_FLAG(RCC_FLAG_LSIRDY) == RESET)
 8000992:	4d5b      	ldr	r5, [pc, #364]	; (8000b00 <HAL_RCC_OscConfig+0x2d4>)
      tickstart = HAL_GetTick();
 8000994:	4606      	mov	r6, r0
      while(__HAL_RCC_GET_FLAG(RCC_FLAG_LSIRDY) == RESET)
 8000996:	6f6b      	ldr	r3, [r5, #116]	; 0x74
 8000998:	079f      	lsls	r7, r3, #30
 800099a:	f53f af59 	bmi.w	8000850 <HAL_RCC_OscConfig+0x24>
        if((HAL_GetTick() - tickstart ) > LSI_TIMEOUT_VALUE)
 800099e:	f7ff fded 	bl	800057c <HAL_GetTick>
 80009a2:	1b80      	subs	r0, r0, r6
 80009a4:	2802      	cmp	r0, #2
 80009a6:	d9f6      	bls.n	8000996 <HAL_RCC_OscConfig+0x16a>
 80009a8:	e787      	b.n	80008ba <HAL_RCC_OscConfig+0x8e>
      __HAL_RCC_LSI_DISABLE();
 80009aa:	601a      	str	r2, [r3, #0]
      tickstart = HAL_GetTick();
 80009ac:	f7ff fde6 	bl	800057c <HAL_GetTick>
      while(__HAL_RCC_GET_FLAG(RCC_FLAG_LSIRDY) != RESET)
 80009b0:	4d53      	ldr	r5, [pc, #332]	; (8000b00 <HAL_RCC_OscConfig+0x2d4>)
      tickstart = HAL_GetTick();
 80009b2:	4606      	mov	r6, r0
      while(__HAL_RCC_GET_FLAG(RCC_FLAG_LSIRDY) != RESET)
 80009b4:	6f6b      	ldr	r3, [r5, #116]	; 0x74
 80009b6:	0798      	lsls	r0, r3, #30
 80009b8:	f57f af4a 	bpl.w	8000850 <HAL_RCC_OscConfig+0x24>
        if((HAL_GetTick() - tickstart ) > LSI_TIMEOUT_VALUE)
 80009bc:	f7ff fdde 	bl	800057c <HAL_GetTick>
 80009c0:	1b80      	subs	r0, r0, r6
 80009c2:	2802      	cmp	r0, #2
 80009c4:	d9f6      	bls.n	80009b4 <HAL_RCC_OscConfig+0x188>
 80009c6:	e778      	b.n	80008ba <HAL_RCC_OscConfig+0x8e>
    if(__HAL_RCC_PWR_IS_CLK_DISABLED())
 80009c8:	4b4d      	ldr	r3, [pc, #308]	; (8000b00 <HAL_RCC_OscConfig+0x2d4>)
 80009ca:	6c1a      	ldr	r2, [r3, #64]	; 0x40
 80009cc:	f012 5280 	ands.w	r2, r2, #268435456	; 0x10000000
 80009d0:	d128      	bne.n	8000a24 <HAL_RCC_OscConfig+0x1f8>
      __HAL_RCC_PWR_CLK_ENABLE();
 80009d2:	9201      	str	r2, [sp, #4]
 80009d4:	6c1a      	ldr	r2, [r3, #64]	; 0x40
 80009d6:	f042 5280 	orr.w	r2, r2, #268435456	; 0x10000000
 80009da:	641a      	str	r2, [r3, #64]	; 0x40
 80009dc:	6c1b      	ldr	r3, [r3, #64]	; 0x40
 80009de:	f003 5380 	and.w	r3, r3, #268435456	; 0x10000000
 80009e2:	9301      	str	r3, [sp, #4]
 80009e4:	9b01      	ldr	r3, [sp, #4]
      pwrclkchanged = SET;
 80009e6:	2601      	movs	r6, #1
    if(HAL_IS_BIT_CLR(PWR->CR, PWR_CR_DBP))
 80009e8:	4d48      	ldr	r5, [pc, #288]	; (8000b0c <HAL_RCC_OscConfig+0x2e0>)
 80009ea:	682b      	ldr	r3, [r5, #0]
 80009ec:	05d9      	lsls	r1, r3, #23
 80009ee:	d51b      	bpl.n	8000a28 <HAL_RCC_OscConfig+0x1fc>
    __HAL_RCC_LSE_CONFIG(RCC_OscInitStruct->LSEState);
 80009f0:	68a3      	ldr	r3, [r4, #8]
 80009f2:	4d43      	ldr	r5, [pc, #268]	; (8000b00 <HAL_RCC_OscConfig+0x2d4>)
 80009f4:	2b01      	cmp	r3, #1
 80009f6:	d127      	bne.n	8000a48 <HAL_RCC_OscConfig+0x21c>
 80009f8:	6f2b      	ldr	r3, [r5, #112]	; 0x70
 80009fa:	f043 0301 	orr.w	r3, r3, #1
 80009fe:	672b      	str	r3, [r5, #112]	; 0x70
      tickstart = HAL_GetTick();
 8000a00:	f7ff fdbc 	bl	800057c <HAL_GetTick>
      while(__HAL_RCC_GET_FLAG(RCC_FLAG_LSERDY) == RESET)
 8000a04:	4d3e      	ldr	r5, [pc, #248]	; (8000b00 <HAL_RCC_OscConfig+0x2d4>)
      tickstart = HAL_GetTick();
 8000a06:	4607      	mov	r7, r0
        if((HAL_GetTick() - tickstart ) > RCC_LSE_TIMEOUT_VALUE)
 8000a08:	f241 3888 	movw	r8, #5000	; 0x1388
      while(__HAL_RCC_GET_FLAG(RCC_FLAG_LSERDY) == RESET)
 8000a0c:	6f2b      	ldr	r3, [r5, #112]	; 0x70
 8000a0e:	079b      	lsls	r3, r3, #30
 8000a10:	d539      	bpl.n	8000a86 <HAL_RCC_OscConfig+0x25a>
    if(pwrclkchanged == SET)
 8000a12:	2e00      	cmp	r6, #0
 8000a14:	f43f af20 	beq.w	8000858 <HAL_RCC_OscConfig+0x2c>
      __HAL_RCC_PWR_CLK_DISABLE();
 8000a18:	4a39      	ldr	r2, [pc, #228]	; (8000b00 <HAL_RCC_OscConfig+0x2d4>)
 8000a1a:	6c13      	ldr	r3, [r2, #64]	; 0x40
 8000a1c:	f023 5380 	bic.w	r3, r3, #268435456	; 0x10000000
 8000a20:	6413      	str	r3, [r2, #64]	; 0x40
 8000a22:	e719      	b.n	8000858 <HAL_RCC_OscConfig+0x2c>
    FlagStatus       pwrclkchanged = RESET;
 8000a24:	2600      	movs	r6, #0
 8000a26:	e7df      	b.n	80009e8 <HAL_RCC_OscConfig+0x1bc>
      SET_BIT(PWR->CR, PWR_CR_DBP);
 8000a28:	682b      	ldr	r3, [r5, #0]
 8000a2a:	f443 7380 	orr.w	r3, r3, #256	; 0x100
 8000a2e:	602b      	str	r3, [r5, #0]
      tickstart = HAL_GetTick();
 8000a30:	f7ff fda4 	bl	800057c <HAL_GetTick>
 8000a34:	4607      	mov	r7, r0
      while(HAL_IS_BIT_CLR(PWR->CR, PWR_CR_DBP))
 8000a36:	682b      	ldr	r3, [r5, #0]
 8000a38:	05da      	lsls	r2, r3, #23
 8000a3a:	d4d9      	bmi.n	80009f0 <HAL_RCC_OscConfig+0x1c4>
        if((HAL_GetTick() - tickstart) > RCC_DBP_TIMEOUT_VALUE)
 8000a3c:	f7ff fd9e 	bl	800057c <HAL_GetTick>
 8000a40:	1bc0      	subs	r0, r0, r7
 8000a42:	2802      	cmp	r0, #2
 8000a44:	d9f7      	bls.n	8000a36 <HAL_RCC_OscConfig+0x20a>
 8000a46:	e738      	b.n	80008ba <HAL_RCC_OscConfig+0x8e>
    __HAL_RCC_LSE_CONFIG(RCC_OscInitStruct->LSEState);
 8000a48:	2b05      	cmp	r3, #5
 8000a4a:	d104      	bne.n	8000a56 <HAL_RCC_OscConfig+0x22a>
 8000a4c:	6f2b      	ldr	r3, [r5, #112]	; 0x70
 8000a4e:	f043 0304 	orr.w	r3, r3, #4
 8000a52:	672b      	str	r3, [r5, #112]	; 0x70
 8000a54:	e7d0      	b.n	80009f8 <HAL_RCC_OscConfig+0x1cc>
 8000a56:	6f2a      	ldr	r2, [r5, #112]	; 0x70
 8000a58:	f022 0201 	bic.w	r2, r2, #1
 8000a5c:	672a      	str	r2, [r5, #112]	; 0x70
 8000a5e:	6f2a      	ldr	r2, [r5, #112]	; 0x70
 8000a60:	f022 0204 	bic.w	r2, r2, #4
 8000a64:	672a      	str	r2, [r5, #112]	; 0x70
    if((RCC_OscInitStruct->LSEState) != RCC_LSE_OFF)
 8000a66:	2b00      	cmp	r3, #0
 8000a68:	d1ca      	bne.n	8000a00 <HAL_RCC_OscConfig+0x1d4>
      tickstart = HAL_GetTick();
 8000a6a:	f7ff fd87 	bl	800057c <HAL_GetTick>
        if((HAL_GetTick() - tickstart ) > RCC_LSE_TIMEOUT_VALUE)
 8000a6e:	f241 3888 	movw	r8, #5000	; 0x1388
      tickstart = HAL_GetTick();
 8000a72:	4607      	mov	r7, r0
      while(__HAL_RCC_GET_FLAG(RCC_FLAG_LSERDY) != RESET)
 8000a74:	6f2b      	ldr	r3, [r5, #112]	; 0x70
 8000a76:	0798      	lsls	r0, r3, #30
 8000a78:	d5cb      	bpl.n	8000a12 <HAL_RCC_OscConfig+0x1e6>
        if((HAL_GetTick() - tickstart ) > RCC_LSE_TIMEOUT_VALUE)
 8000a7a:	f7ff fd7f 	bl	800057c <HAL_GetTick>
 8000a7e:	1bc0      	subs	r0, r0, r7
 8000a80:	4540      	cmp	r0, r8
 8000a82:	d9f7      	bls.n	8000a74 <HAL_RCC_OscConfig+0x248>
 8000a84:	e719      	b.n	80008ba <HAL_RCC_OscConfig+0x8e>
        if((HAL_GetTick() - tickstart ) > RCC_LSE_TIMEOUT_VALUE)
 8000a86:	f7ff fd79 	bl	800057c <HAL_GetTick>
 8000a8a:	1bc0      	subs	r0, r0, r7
 8000a8c:	4540      	cmp	r0, r8
 8000a8e:	d9bd      	bls.n	8000a0c <HAL_RCC_OscConfig+0x1e0>
 8000a90:	e713      	b.n	80008ba <HAL_RCC_OscConfig+0x8e>
    if(__HAL_RCC_GET_SYSCLK_SOURCE() != RCC_CFGR_SWS_PLL)
 8000a92:	4d1b      	ldr	r5, [pc, #108]	; (8000b00 <HAL_RCC_OscConfig+0x2d4>)
 8000a94:	68ab      	ldr	r3, [r5, #8]
 8000a96:	f003 030c 	and.w	r3, r3, #12
 8000a9a:	2b08      	cmp	r3, #8
 8000a9c:	f43f aeca 	beq.w	8000834 <HAL_RCC_OscConfig+0x8>
 8000aa0:	4e1b      	ldr	r6, [pc, #108]	; (8000b10 <HAL_RCC_OscConfig+0x2e4>)
 8000aa2:	2300      	movs	r3, #0
      if((RCC_OscInitStruct->PLL.PLLState) == RCC_PLL_ON)
 8000aa4:	2a02      	cmp	r2, #2
        __HAL_RCC_PLL_DISABLE();
 8000aa6:	6033      	str	r3, [r6, #0]
      if((RCC_OscInitStruct->PLL.PLLState) == RCC_PLL_ON)
 8000aa8:	d134      	bne.n	8000b14 <HAL_RCC_OscConfig+0x2e8>
        tickstart = HAL_GetTick();
 8000aaa:	f7ff fd67 	bl	800057c <HAL_GetTick>
 8000aae:	4607      	mov	r7, r0
        while(__HAL_RCC_GET_FLAG(RCC_FLAG_PLLRDY) != RESET)
 8000ab0:	682b      	ldr	r3, [r5, #0]
 8000ab2:	0199      	lsls	r1, r3, #6
 8000ab4:	d41e      	bmi.n	8000af4 <HAL_RCC_OscConfig+0x2c8>
        WRITE_REG(RCC->PLLCFGR, (RCC_OscInitStruct->PLL.PLLSource                                            | \
 8000ab6:	6a22      	ldr	r2, [r4, #32]
 8000ab8:	69e3      	ldr	r3, [r4, #28]
 8000aba:	4313      	orrs	r3, r2
 8000abc:	6a62      	ldr	r2, [r4, #36]	; 0x24
 8000abe:	ea43 1382 	orr.w	r3, r3, r2, lsl #6
 8000ac2:	6ae2      	ldr	r2, [r4, #44]	; 0x2c
 8000ac4:	ea43 6302 	orr.w	r3, r3, r2, lsl #24
 8000ac8:	6aa2      	ldr	r2, [r4, #40]	; 0x28
        while(__HAL_RCC_GET_FLAG(RCC_FLAG_PLLRDY) == RESET)
 8000aca:	4c0d      	ldr	r4, [pc, #52]	; (8000b00 <HAL_RCC_OscConfig+0x2d4>)
        WRITE_REG(RCC->PLLCFGR, (RCC_OscInitStruct->PLL.PLLSource                                            | \
 8000acc:	0852      	lsrs	r2, r2, #1
 8000ace:	3a01      	subs	r2, #1
 8000ad0:	ea43 4302 	orr.w	r3, r3, r2, lsl #16
 8000ad4:	606b      	str	r3, [r5, #4]
        __HAL_RCC_PLL_ENABLE();
 8000ad6:	2301      	movs	r3, #1
 8000ad8:	6033      	str	r3, [r6, #0]
        tickstart = HAL_GetTick();
 8000ada:	f7ff fd4f 	bl	800057c <HAL_GetTick>
 8000ade:	4605      	mov	r5, r0
        while(__HAL_RCC_GET_FLAG(RCC_FLAG_PLLRDY) == RESET)
 8000ae0:	6823      	ldr	r3, [r4, #0]
 8000ae2:	019a      	lsls	r2, r3, #6
 8000ae4:	f53f aebc 	bmi.w	8000860 <HAL_RCC_OscConfig+0x34>
          if((HAL_GetTick() - tickstart ) > PLL_TIMEOUT_VALUE)
 8000ae8:	f7ff fd48 	bl	800057c <HAL_GetTick>
 8000aec:	1b40      	subs	r0, r0, r5
 8000aee:	2802      	cmp	r0, #2
 8000af0:	d9f6      	bls.n	8000ae0 <HAL_RCC_OscConfig+0x2b4>
 8000af2:	e6e2      	b.n	80008ba <HAL_RCC_OscConfig+0x8e>
          if((HAL_GetTick() - tickstart ) > PLL_TIMEOUT_VALUE)
 8000af4:	f7ff fd42 	bl	800057c <HAL_GetTick>
 8000af8:	1bc0      	subs	r0, r0, r7
 8000afa:	2802      	cmp	r0, #2
 8000afc:	d9d8      	bls.n	8000ab0 <HAL_RCC_OscConfig+0x284>
 8000afe:	e6dc      	b.n	80008ba <HAL_RCC_OscConfig+0x8e>
 8000b00:	40023800 	.word	0x40023800
 8000b04:	42470000 	.word	0x42470000
 8000b08:	42470e80 	.word	0x42470e80
 8000b0c:	40007000 	.word	0x40007000
 8000b10:	42470060 	.word	0x42470060
        tickstart = HAL_GetTick();
 8000b14:	f7ff fd32 	bl	800057c <HAL_GetTick>
 8000b18:	4604      	mov	r4, r0
        while(__HAL_RCC_GET_FLAG(RCC_FLAG_PLLRDY) != RESET)
 8000b1a:	682b      	ldr	r3, [r5, #0]
 8000b1c:	019b      	lsls	r3, r3, #6
 8000b1e:	f57f ae9f 	bpl.w	8000860 <HAL_RCC_OscConfig+0x34>
          if((HAL_GetTick() - tickstart ) > PLL_TIMEOUT_VALUE)
 8000b22:	f7ff fd2b 	bl	800057c <HAL_GetTick>
 8000b26:	1b00      	subs	r0, r0, r4
 8000b28:	2802      	cmp	r0, #2
 8000b2a:	d9f6      	bls.n	8000b1a <HAL_RCC_OscConfig+0x2ee>
 8000b2c:	e6c5      	b.n	80008ba <HAL_RCC_OscConfig+0x8e>
 8000b2e:	bf00      	nop

08000b30 <HAL_RCC_GetSysClockFreq>:
{
  uint32_t pllm = 0U, pllvco = 0U, pllp = 0U;
  uint32_t sysclockfreq = 0U;

  /* Get SYSCLK source -------------------------------------------------------*/
  switch (RCC->CFGR & RCC_CFGR_SWS)
 8000b30:	4913      	ldr	r1, [pc, #76]	; (8000b80 <HAL_RCC_GetSysClockFreq+0x50>)
{
 8000b32:	b508      	push	{r3, lr}
  switch (RCC->CFGR & RCC_CFGR_SWS)
 8000b34:	688b      	ldr	r3, [r1, #8]
 8000b36:	f003 030c 	and.w	r3, r3, #12
 8000b3a:	2b04      	cmp	r3, #4
 8000b3c:	d003      	beq.n	8000b46 <HAL_RCC_GetSysClockFreq+0x16>
 8000b3e:	2b08      	cmp	r3, #8
 8000b40:	d003      	beq.n	8000b4a <HAL_RCC_GetSysClockFreq+0x1a>
  {
    case RCC_CFGR_SWS_HSI:  /* HSI used as system clock source */
    {
      sysclockfreq = HSI_VALUE;
 8000b42:	4810      	ldr	r0, [pc, #64]	; (8000b84 <HAL_RCC_GetSysClockFreq+0x54>)
      sysclockfreq = HSI_VALUE;
      break;
    }
  }
  return sysclockfreq;
}
 8000b44:	bd08      	pop	{r3, pc}
      sysclockfreq = HSE_VALUE;
 8000b46:	4810      	ldr	r0, [pc, #64]	; (8000b88 <HAL_RCC_GetSysClockFreq+0x58>)
 8000b48:	bd08      	pop	{r3, pc}
      pllm = RCC->PLLCFGR & RCC_PLLCFGR_PLLM;
 8000b4a:	684a      	ldr	r2, [r1, #4]
      if(__HAL_RCC_GET_PLL_OSCSOURCE() != RCC_PLLSOURCE_HSI)
 8000b4c:	684b      	ldr	r3, [r1, #4]
        pllvco = (uint32_t) ((((uint64_t) HSE_VALUE * ((uint64_t) ((RCC->PLLCFGR & RCC_PLLCFGR_PLLN) >> RCC_PLLCFGR_PLLN_Pos)))) / (uint64_t)pllm);
 8000b4e:	6849      	ldr	r1, [r1, #4]
      if(__HAL_RCC_GET_PLL_OSCSOURCE() != RCC_PLLSOURCE_HSI)
 8000b50:	f413 0380 	ands.w	r3, r3, #4194304	; 0x400000
        pllvco = (uint32_t) ((((uint64_t) HSE_VALUE * ((uint64_t) ((RCC->PLLCFGR & RCC_PLLCFGR_PLLN) >> RCC_PLLCFGR_PLLN_Pos)))) / (uint64_t)pllm);
 8000b54:	bf14      	ite	ne
 8000b56:	480c      	ldrne	r0, [pc, #48]	; (8000b88 <HAL_RCC_GetSysClockFreq+0x58>)
        pllvco = (uint32_t) ((((uint64_t) HSI_VALUE * ((uint64_t) ((RCC->PLLCFGR & RCC_PLLCFGR_PLLN) >> RCC_PLLCFGR_PLLN_Pos)))) / (uint64_t)pllm);
 8000b58:	480a      	ldreq	r0, [pc, #40]	; (8000b84 <HAL_RCC_GetSysClockFreq+0x54>)
        pllvco = (uint32_t) ((((uint64_t) HSE_VALUE * ((uint64_t) ((RCC->PLLCFGR & RCC_PLLCFGR_PLLN) >> RCC_PLLCFGR_PLLN_Pos)))) / (uint64_t)pllm);
 8000b5a:	f3c1 1188 	ubfx	r1, r1, #6, #9
 8000b5e:	bf18      	it	ne
 8000b60:	2300      	movne	r3, #0
      pllm = RCC->PLLCFGR & RCC_PLLCFGR_PLLM;
 8000b62:	f002 023f 	and.w	r2, r2, #63	; 0x3f
        pllvco = (uint32_t) ((((uint64_t) HSI_VALUE * ((uint64_t) ((RCC->PLLCFGR & RCC_PLLCFGR_PLLN) >> RCC_PLLCFGR_PLLN_Pos)))) / (uint64_t)pllm);
 8000b66:	fba1 0100 	umull	r0, r1, r1, r0
 8000b6a:	f7ff fb35 	bl	80001d8 <__aeabi_uldivmod>
      pllp = ((((RCC->PLLCFGR & RCC_PLLCFGR_PLLP) >> RCC_PLLCFGR_PLLP_Pos) + 1U) *2U);
 8000b6e:	4b04      	ldr	r3, [pc, #16]	; (8000b80 <HAL_RCC_GetSysClockFreq+0x50>)
 8000b70:	685b      	ldr	r3, [r3, #4]
 8000b72:	f3c3 4301 	ubfx	r3, r3, #16, #2
 8000b76:	3301      	adds	r3, #1
 8000b78:	005b      	lsls	r3, r3, #1
      sysclockfreq = pllvco/pllp;
 8000b7a:	fbb0 f0f3 	udiv	r0, r0, r3
 8000b7e:	bd08      	pop	{r3, pc}
 8000b80:	40023800 	.word	0x40023800
 8000b84:	00f42400 	.word	0x00f42400
 8000b88:	007a1200 	.word	0x007a1200

08000b8c <HAL_RCC_ClockConfig>:
{
 8000b8c:	e92d 41f0 	stmdb	sp!, {r4, r5, r6, r7, r8, lr}
 8000b90:	460d      	mov	r5, r1
  if(RCC_ClkInitStruct == NULL)
 8000b92:	4604      	mov	r4, r0
 8000b94:	b910      	cbnz	r0, 8000b9c <HAL_RCC_ClockConfig+0x10>
    return HAL_ERROR;
 8000b96:	2001      	movs	r0, #1
 8000b98:	e8bd 81f0 	ldmia.w	sp!, {r4, r5, r6, r7, r8, pc}
  if(FLatency > __HAL_FLASH_GET_LATENCY())
 8000b9c:	4b44      	ldr	r3, [pc, #272]	; (8000cb0 <HAL_RCC_ClockConfig+0x124>)
 8000b9e:	681a      	ldr	r2, [r3, #0]
 8000ba0:	f002 020f 	and.w	r2, r2, #15
 8000ba4:	428a      	cmp	r2, r1
 8000ba6:	d328      	bcc.n	8000bfa <HAL_RCC_ClockConfig+0x6e>
  if(((RCC_ClkInitStruct->ClockType) & RCC_CLOCKTYPE_HCLK) == RCC_CLOCKTYPE_HCLK)
 8000ba8:	6821      	ldr	r1, [r4, #0]
 8000baa:	078f      	lsls	r7, r1, #30
 8000bac:	d42d      	bmi.n	8000c0a <HAL_RCC_ClockConfig+0x7e>
  if(((RCC_ClkInitStruct->ClockType) & RCC_CLOCKTYPE_SYSCLK) == RCC_CLOCKTYPE_SYSCLK)
 8000bae:	07c8      	lsls	r0, r1, #31
 8000bb0:	d440      	bmi.n	8000c34 <HAL_RCC_ClockConfig+0xa8>
  if(FLatency < __HAL_FLASH_GET_LATENCY())
 8000bb2:	4b3f      	ldr	r3, [pc, #252]	; (8000cb0 <HAL_RCC_ClockConfig+0x124>)
 8000bb4:	681a      	ldr	r2, [r3, #0]
 8000bb6:	f002 020f 	and.w	r2, r2, #15
 8000bba:	4295      	cmp	r5, r2
 8000bbc:	d366      	bcc.n	8000c8c <HAL_RCC_ClockConfig+0x100>
  if(((RCC_ClkInitStruct->ClockType) & RCC_CLOCKTYPE_PCLK1) == RCC_CLOCKTYPE_PCLK1)
 8000bbe:	6822      	ldr	r2, [r4, #0]
 8000bc0:	0751      	lsls	r1, r2, #29
 8000bc2:	d46c      	bmi.n	8000c9e <HAL_RCC_ClockConfig+0x112>
  if(((RCC_ClkInitStruct->ClockType) & RCC_CLOCKTYPE_PCLK2) == RCC_CLOCKTYPE_PCLK2)
 8000bc4:	0713      	lsls	r3, r2, #28
 8000bc6:	d507      	bpl.n	8000bd8 <HAL_RCC_ClockConfig+0x4c>
    MODIFY_REG(RCC->CFGR, RCC_CFGR_PPRE2, ((RCC_ClkInitStruct->APB2CLKDivider) << 3U));
 8000bc8:	4a3a      	ldr	r2, [pc, #232]	; (8000cb4 <HAL_RCC_ClockConfig+0x128>)
 8000bca:	6921      	ldr	r1, [r4, #16]
 8000bcc:	6893      	ldr	r3, [r2, #8]
 8000bce:	f423 4360 	bic.w	r3, r3, #57344	; 0xe000
 8000bd2:	ea43 03c1 	orr.w	r3, r3, r1, lsl #3
 8000bd6:	6093      	str	r3, [r2, #8]
  SystemCoreClock = HAL_RCC_GetSysClockFreq() >> AHBPrescTable[(RCC->CFGR & RCC_CFGR_HPRE)>> RCC_CFGR_HPRE_Pos];
 8000bd8:	f7ff ffaa 	bl	8000b30 <HAL_RCC_GetSysClockFreq>
 8000bdc:	4b35      	ldr	r3, [pc, #212]	; (8000cb4 <HAL_RCC_ClockConfig+0x128>)
 8000bde:	4a36      	ldr	r2, [pc, #216]	; (8000cb8 <HAL_RCC_ClockConfig+0x12c>)
 8000be0:	689b      	ldr	r3, [r3, #8]
 8000be2:	f3c3 1303 	ubfx	r3, r3, #4, #4
 8000be6:	5cd3      	ldrb	r3, [r2, r3]
 8000be8:	40d8      	lsrs	r0, r3
 8000bea:	4b34      	ldr	r3, [pc, #208]	; (8000cbc <HAL_RCC_ClockConfig+0x130>)
 8000bec:	6018      	str	r0, [r3, #0]
  HAL_InitTick (TICK_INT_PRIORITY);
 8000bee:	2000      	movs	r0, #0
 8000bf0:	f7ff fc7a 	bl	80004e8 <HAL_InitTick>
  return HAL_OK;
 8000bf4:	2000      	movs	r0, #0
 8000bf6:	e8bd 81f0 	ldmia.w	sp!, {r4, r5, r6, r7, r8, pc}
    __HAL_FLASH_SET_LATENCY(FLatency);
 8000bfa:	b2ca      	uxtb	r2, r1
 8000bfc:	701a      	strb	r2, [r3, #0]
    if(__HAL_FLASH_GET_LATENCY() != FLatency)
 8000bfe:	681b      	ldr	r3, [r3, #0]
 8000c00:	f003 030f 	and.w	r3, r3, #15
 8000c04:	4299      	cmp	r1, r3
 8000c06:	d1c6      	bne.n	8000b96 <HAL_RCC_ClockConfig+0xa>
 8000c08:	e7ce      	b.n	8000ba8 <HAL_RCC_ClockConfig+0x1c>
 8000c0a:	4b2a      	ldr	r3, [pc, #168]	; (8000cb4 <HAL_RCC_ClockConfig+0x128>)
    if(((RCC_ClkInitStruct->ClockType) & RCC_CLOCKTYPE_PCLK1) == RCC_CLOCKTYPE_PCLK1)
 8000c0c:	f011 0f04 	tst.w	r1, #4
      MODIFY_REG(RCC->CFGR, RCC_CFGR_PPRE1, RCC_HCLK_DIV16);
 8000c10:	bf1e      	ittt	ne
 8000c12:	689a      	ldrne	r2, [r3, #8]
 8000c14:	f442 52e0 	orrne.w	r2, r2, #7168	; 0x1c00
 8000c18:	609a      	strne	r2, [r3, #8]
    if(((RCC_ClkInitStruct->ClockType) & RCC_CLOCKTYPE_PCLK2) == RCC_CLOCKTYPE_PCLK2)
 8000c1a:	070e      	lsls	r6, r1, #28
      MODIFY_REG(RCC->CFGR, RCC_CFGR_PPRE2, (RCC_HCLK_DIV16 << 3));
 8000c1c:	bf42      	ittt	mi
 8000c1e:	689a      	ldrmi	r2, [r3, #8]
 8000c20:	f442 4260 	orrmi.w	r2, r2, #57344	; 0xe000
 8000c24:	609a      	strmi	r2, [r3, #8]
    MODIFY_REG(RCC->CFGR, RCC_CFGR_HPRE, RCC_ClkInitStruct->AHBCLKDivider);
 8000c26:	689a      	ldr	r2, [r3, #8]
 8000c28:	68a0      	ldr	r0, [r4, #8]
 8000c2a:	f022 02f0 	bic.w	r2, r2, #240	; 0xf0
 8000c2e:	4302      	orrs	r2, r0
 8000c30:	609a      	str	r2, [r3, #8]
 8000c32:	e7bc      	b.n	8000bae <HAL_RCC_ClockConfig+0x22>
    if(RCC_ClkInitStruct->SYSCLKSource == RCC_SYSCLKSOURCE_HSE)
 8000c34:	6862      	ldr	r2, [r4, #4]
 8000c36:	4b1f      	ldr	r3, [pc, #124]	; (8000cb4 <HAL_RCC_ClockConfig+0x128>)
 8000c38:	2a01      	cmp	r2, #1
 8000c3a:	d11d      	bne.n	8000c78 <HAL_RCC_ClockConfig+0xec>
      if(__HAL_RCC_GET_FLAG(RCC_FLAG_HSERDY) == RESET)
 8000c3c:	681b      	ldr	r3, [r3, #0]
 8000c3e:	f413 3f00 	tst.w	r3, #131072	; 0x20000
      if(__HAL_RCC_GET_FLAG(RCC_FLAG_HSIRDY) == RESET)
 8000c42:	d0a8      	beq.n	8000b96 <HAL_RCC_ClockConfig+0xa>
    __HAL_RCC_SYSCLK_CONFIG(RCC_ClkInitStruct->SYSCLKSource);
 8000c44:	4e1b      	ldr	r6, [pc, #108]	; (8000cb4 <HAL_RCC_ClockConfig+0x128>)
 8000c46:	68b3      	ldr	r3, [r6, #8]
 8000c48:	f023 0303 	bic.w	r3, r3, #3
 8000c4c:	4313      	orrs	r3, r2
 8000c4e:	60b3      	str	r3, [r6, #8]
    tickstart = HAL_GetTick();
 8000c50:	f7ff fc94 	bl	800057c <HAL_GetTick>
      if ((HAL_GetTick() - tickstart) > CLOCKSWITCH_TIMEOUT_VALUE)
 8000c54:	f241 3888 	movw	r8, #5000	; 0x1388
    tickstart = HAL_GetTick();
 8000c58:	4607      	mov	r7, r0
    while (__HAL_RCC_GET_SYSCLK_SOURCE() != (RCC_ClkInitStruct->SYSCLKSource << RCC_CFGR_SWS_Pos))
 8000c5a:	68b3      	ldr	r3, [r6, #8]
 8000c5c:	6862      	ldr	r2, [r4, #4]
 8000c5e:	f003 030c 	and.w	r3, r3, #12
 8000c62:	ebb3 0f82 	cmp.w	r3, r2, lsl #2
 8000c66:	d0a4      	beq.n	8000bb2 <HAL_RCC_ClockConfig+0x26>
      if ((HAL_GetTick() - tickstart) > CLOCKSWITCH_TIMEOUT_VALUE)
 8000c68:	f7ff fc88 	bl	800057c <HAL_GetTick>
 8000c6c:	1bc0      	subs	r0, r0, r7
 8000c6e:	4540      	cmp	r0, r8
 8000c70:	d9f3      	bls.n	8000c5a <HAL_RCC_ClockConfig+0xce>
        return HAL_TIMEOUT;
 8000c72:	2003      	movs	r0, #3
}
 8000c74:	e8bd 81f0 	ldmia.w	sp!, {r4, r5, r6, r7, r8, pc}
    else if((RCC_ClkInitStruct->SYSCLKSource == RCC_SYSCLKSOURCE_PLLCLK)   ||
 8000c78:	1e91      	subs	r1, r2, #2
 8000c7a:	2901      	cmp	r1, #1
      if(__HAL_RCC_GET_FLAG(RCC_FLAG_PLLRDY) == RESET)
 8000c7c:	681b      	ldr	r3, [r3, #0]
    else if((RCC_ClkInitStruct->SYSCLKSource == RCC_SYSCLKSOURCE_PLLCLK)   ||
 8000c7e:	d802      	bhi.n	8000c86 <HAL_RCC_ClockConfig+0xfa>
      if(__HAL_RCC_GET_FLAG(RCC_FLAG_PLLRDY) == RESET)
 8000c80:	f013 7f00 	tst.w	r3, #33554432	; 0x2000000
 8000c84:	e7dd      	b.n	8000c42 <HAL_RCC_ClockConfig+0xb6>
      if(__HAL_RCC_GET_FLAG(RCC_FLAG_HSIRDY) == RESET)
 8000c86:	f013 0f02 	tst.w	r3, #2
 8000c8a:	e7da      	b.n	8000c42 <HAL_RCC_ClockConfig+0xb6>
    __HAL_FLASH_SET_LATENCY(FLatency);
 8000c8c:	b2ea      	uxtb	r2, r5
 8000c8e:	701a      	strb	r2, [r3, #0]
    if(__HAL_FLASH_GET_LATENCY() != FLatency)
 8000c90:	681b      	ldr	r3, [r3, #0]
 8000c92:	f003 030f 	and.w	r3, r3, #15
 8000c96:	429d      	cmp	r5, r3
 8000c98:	f47f af7d 	bne.w	8000b96 <HAL_RCC_ClockConfig+0xa>
 8000c9c:	e78f      	b.n	8000bbe <HAL_RCC_ClockConfig+0x32>
    MODIFY_REG(RCC->CFGR, RCC_CFGR_PPRE1, RCC_ClkInitStruct->APB1CLKDivider);
 8000c9e:	4905      	ldr	r1, [pc, #20]	; (8000cb4 <HAL_RCC_ClockConfig+0x128>)
 8000ca0:	68e0      	ldr	r0, [r4, #12]
 8000ca2:	688b      	ldr	r3, [r1, #8]
 8000ca4:	f423 53e0 	bic.w	r3, r3, #7168	; 0x1c00
 8000ca8:	4303      	orrs	r3, r0
 8000caa:	608b      	str	r3, [r1, #8]
 8000cac:	e78a      	b.n	8000bc4 <HAL_RCC_ClockConfig+0x38>
 8000cae:	bf00      	nop
 8000cb0:	40023c00 	.word	0x40023c00
 8000cb4:	40023800 	.word	0x40023800
 8000cb8:	080012dc 	.word	0x080012dc
 8000cbc:	20000008 	.word	0x20000008

08000cc0 <HAL_RCC_GetPCLK1Freq>:
  * @retval PCLK1 frequency
  */
uint32_t HAL_RCC_GetPCLK1Freq(void)
{
  /* Get HCLK source and Compute PCLK1 frequency ---------------------------*/
  return (HAL_RCC_GetHCLKFreq() >> APBPrescTable[(RCC->CFGR & RCC_CFGR_PPRE1)>> RCC_CFGR_PPRE1_Pos]);
 8000cc0:	4b04      	ldr	r3, [pc, #16]	; (8000cd4 <HAL_RCC_GetPCLK1Freq+0x14>)
 8000cc2:	4a05      	ldr	r2, [pc, #20]	; (8000cd8 <HAL_RCC_GetPCLK1Freq+0x18>)
 8000cc4:	689b      	ldr	r3, [r3, #8]
 8000cc6:	f3c3 2382 	ubfx	r3, r3, #10, #3
 8000cca:	5cd3      	ldrb	r3, [r2, r3]
 8000ccc:	4a03      	ldr	r2, [pc, #12]	; (8000cdc <HAL_RCC_GetPCLK1Freq+0x1c>)
 8000cce:	6810      	ldr	r0, [r2, #0]
}
 8000cd0:	40d8      	lsrs	r0, r3
 8000cd2:	4770      	bx	lr
 8000cd4:	40023800 	.word	0x40023800
 8000cd8:	080012ec 	.word	0x080012ec
 8000cdc:	20000008 	.word	0x20000008

08000ce0 <HAL_RCC_GetPCLK2Freq>:
  * @retval PCLK2 frequency
  */
uint32_t HAL_RCC_GetPCLK2Freq(void)
{
  /* Get HCLK source and Compute PCLK2 frequency ---------------------------*/
  return (HAL_RCC_GetHCLKFreq()>> APBPrescTable[(RCC->CFGR & RCC_CFGR_PPRE2)>> RCC_CFGR_PPRE2_Pos]);
 8000ce0:	4b04      	ldr	r3, [pc, #16]	; (8000cf4 <HAL_RCC_GetPCLK2Freq+0x14>)
 8000ce2:	4a05      	ldr	r2, [pc, #20]	; (8000cf8 <HAL_RCC_GetPCLK2Freq+0x18>)
 8000ce4:	689b      	ldr	r3, [r3, #8]
 8000ce6:	f3c3 3342 	ubfx	r3, r3, #13, #3
 8000cea:	5cd3      	ldrb	r3, [r2, r3]
 8000cec:	4a03      	ldr	r2, [pc, #12]	; (8000cfc <HAL_RCC_GetPCLK2Freq+0x1c>)
 8000cee:	6810      	ldr	r0, [r2, #0]
}
 8000cf0:	40d8      	lsrs	r0, r3
 8000cf2:	4770      	bx	lr
 8000cf4:	40023800 	.word	0x40023800
 8000cf8:	080012ec 	.word	0x080012ec
 8000cfc:	20000008 	.word	0x20000008

08000d00 <UART_SetConfig>:
  * @param  huart  Pointer to a UART_HandleTypeDef structure that contains
  *                the configuration information for the specified UART module.
  * @retval None
  */
static void UART_SetConfig(UART_HandleTypeDef *huart)
{
 8000d00:	e92d 47f0 	stmdb	sp!, {r4, r5, r6, r7, r8, r9, sl, lr}
  assert_param(IS_UART_MODE(huart->Init.Mode));

  /*-------------------------- USART CR2 Configuration -----------------------*/
  /* Configure the UART Stop Bits: Set STOP[13:12] bits
     according to huart->Init.StopBits value */
  MODIFY_REG(huart->Instance->CR2, USART_CR2_STOP, huart->Init.StopBits);
 8000d04:	6806      	ldr	r6, [r0, #0]
 8000d06:	68c2      	ldr	r2, [r0, #12]
 8000d08:	6933      	ldr	r3, [r6, #16]
     Set the M bits according to huart->Init.WordLength value
     Set PCE and PS bits according to huart->Init.Parity value
     Set TE and RE bits according to huart->Init.Mode value
     Set OVER8 bit according to huart->Init.OverSampling value */

  tmpreg = (uint32_t)huart->Init.WordLength | huart->Init.Parity | huart->Init.Mode | huart->Init.OverSampling;
 8000d0a:	69c1      	ldr	r1, [r0, #28]
  MODIFY_REG(huart->Instance->CR2, USART_CR2_STOP, huart->Init.StopBits);
 8000d0c:	f423 5340 	bic.w	r3, r3, #12288	; 0x3000
 8000d10:	4313      	orrs	r3, r2
 8000d12:	6133      	str	r3, [r6, #16]
{
 8000d14:	4604      	mov	r4, r0
  tmpreg = (uint32_t)huart->Init.WordLength | huart->Init.Parity | huart->Init.Mode | huart->Init.OverSampling;
 8000d16:	6883      	ldr	r3, [r0, #8]
 8000d18:	6900      	ldr	r0, [r0, #16]
  MODIFY_REG(huart->Instance->CR1,
 8000d1a:	68f2      	ldr	r2, [r6, #12]
  tmpreg = (uint32_t)huart->Init.WordLength | huart->Init.Parity | huart->Init.Mode | huart->Init.OverSampling;
 8000d1c:	4303      	orrs	r3, r0
 8000d1e:	6960      	ldr	r0, [r4, #20]
  MODIFY_REG(huart->Instance->CR1,
 8000d20:	f422 4216 	bic.w	r2, r2, #38400	; 0x9600
  tmpreg = (uint32_t)huart->Init.WordLength | huart->Init.Parity | huart->Init.Mode | huart->Init.OverSampling;
 8000d24:	4303      	orrs	r3, r0
  MODIFY_REG(huart->Instance->CR1,
 8000d26:	f022 020c 	bic.w	r2, r2, #12
  tmpreg = (uint32_t)huart->Init.WordLength | huart->Init.Parity | huart->Init.Mode | huart->Init.OverSampling;
 8000d2a:	430b      	orrs	r3, r1
  MODIFY_REG(huart->Instance->CR1,
 8000d2c:	4313      	orrs	r3, r2
 8000d2e:	60f3      	str	r3, [r6, #12]
             (uint32_t)(USART_CR1_M | USART_CR1_PCE | USART_CR1_PS | USART_CR1_TE | USART_CR1_RE | USART_CR1_OVER8),
             tmpreg);

  /*-------------------------- USART CR3 Configuration -----------------------*/
  /* Configure the UART HFC: Set CTSE and RTSE bits according to huart->Init.HwFlowCtl value */
  MODIFY_REG(huart->Instance->CR3, (USART_CR3_RTSE | USART_CR3_CTSE), huart->Init.HwFlowCtl);
 8000d30:	6973      	ldr	r3, [r6, #20]
 8000d32:	69a2      	ldr	r2, [r4, #24]
 8000d34:	f423 7340 	bic.w	r3, r3, #768	; 0x300
 8000d38:	4313      	orrs	r3, r2

  /* Check the Over Sampling */
  if (huart->Init.OverSampling == UART_OVERSAMPLING_8)
 8000d3a:	f5b1 4f00 	cmp.w	r1, #32768	; 0x8000
  MODIFY_REG(huart->Instance->CR3, (USART_CR3_RTSE | USART_CR3_CTSE), huart->Init.HwFlowCtl);
 8000d3e:	6173      	str	r3, [r6, #20]
 8000d40:	4b7a      	ldr	r3, [pc, #488]	; (8000f2c <UART_SetConfig+0x22c>)
  if (huart->Init.OverSampling == UART_OVERSAMPLING_8)
 8000d42:	d17c      	bne.n	8000e3e <UART_SetConfig+0x13e>
  {
    /*-------------------------- USART BRR Configuration ---------------------*/
#if defined(USART6)
    if ((huart->Instance == USART1) || (huart->Instance == USART6))
 8000d44:	429e      	cmp	r6, r3
 8000d46:	d003      	beq.n	8000d50 <UART_SetConfig+0x50>
 8000d48:	f503 6380 	add.w	r3, r3, #1024	; 0x400
 8000d4c:	429e      	cmp	r6, r3
 8000d4e:	d144      	bne.n	8000dda <UART_SetConfig+0xda>
    {
      huart->Instance->BRR = UART_BRR_SAMPLING8(HAL_RCC_GetPCLK2Freq(), huart->Init.BaudRate);
 8000d50:	f7ff ffc6 	bl	8000ce0 <HAL_RCC_GetPCLK2Freq>
 8000d54:	2519      	movs	r5, #25
 8000d56:	fb05 f300 	mul.w	r3, r5, r0
 8000d5a:	6860      	ldr	r0, [r4, #4]
 8000d5c:	f04f 0964 	mov.w	r9, #100	; 0x64
 8000d60:	0040      	lsls	r0, r0, #1
 8000d62:	fbb3 f3f0 	udiv	r3, r3, r0
 8000d66:	fbb3 f3f9 	udiv	r3, r3, r9
 8000d6a:	ea4f 1803 	mov.w	r8, r3, lsl #4
 8000d6e:	f7ff ffb7 	bl	8000ce0 <HAL_RCC_GetPCLK2Freq>
 8000d72:	6863      	ldr	r3, [r4, #4]
 8000d74:	4368      	muls	r0, r5
 8000d76:	005b      	lsls	r3, r3, #1
 8000d78:	fbb0 f7f3 	udiv	r7, r0, r3
 8000d7c:	f7ff ffb0 	bl	8000ce0 <HAL_RCC_GetPCLK2Freq>
 8000d80:	6863      	ldr	r3, [r4, #4]
 8000d82:	4368      	muls	r0, r5
 8000d84:	005b      	lsls	r3, r3, #1
 8000d86:	fbb0 f3f3 	udiv	r3, r0, r3
 8000d8a:	fbb3 f3f9 	udiv	r3, r3, r9
 8000d8e:	fb09 7313 	mls	r3, r9, r3, r7
 8000d92:	00db      	lsls	r3, r3, #3
 8000d94:	3332      	adds	r3, #50	; 0x32
 8000d96:	fbb3 f3f9 	udiv	r3, r3, r9
 8000d9a:	005b      	lsls	r3, r3, #1
 8000d9c:	f403 77f8 	and.w	r7, r3, #496	; 0x1f0
 8000da0:	f7ff ff9e 	bl	8000ce0 <HAL_RCC_GetPCLK2Freq>
 8000da4:	6862      	ldr	r2, [r4, #4]
 8000da6:	4368      	muls	r0, r5
 8000da8:	0052      	lsls	r2, r2, #1
 8000daa:	fbb0 faf2 	udiv	sl, r0, r2
 8000dae:	f7ff ff97 	bl	8000ce0 <HAL_RCC_GetPCLK2Freq>
      huart->Instance->BRR = UART_BRR_SAMPLING8(HAL_RCC_GetPCLK2Freq(), huart->Init.BaudRate);
    }
#endif /* USART6 */
    else
    {
      huart->Instance->BRR = UART_BRR_SAMPLING8(HAL_RCC_GetPCLK1Freq(), huart->Init.BaudRate);
 8000db2:	6863      	ldr	r3, [r4, #4]
 8000db4:	4368      	muls	r0, r5
 8000db6:	005b      	lsls	r3, r3, #1
 8000db8:	fbb0 f3f3 	udiv	r3, r0, r3
 8000dbc:	fbb3 f3f9 	udiv	r3, r3, r9
 8000dc0:	fb09 a313 	mls	r3, r9, r3, sl
 8000dc4:	00db      	lsls	r3, r3, #3
 8000dc6:	3332      	adds	r3, #50	; 0x32
 8000dc8:	fbb3 f3f9 	udiv	r3, r3, r9
 8000dcc:	f003 0307 	and.w	r3, r3, #7
 8000dd0:	4443      	add	r3, r8
      huart->Instance->BRR = UART_BRR_SAMPLING16(HAL_RCC_GetPCLK2Freq(), huart->Init.BaudRate);
    }
#endif /* USART6 */
    else
    {
      huart->Instance->BRR = UART_BRR_SAMPLING16(HAL_RCC_GetPCLK1Freq(), huart->Init.BaudRate);
 8000dd2:	443b      	add	r3, r7
 8000dd4:	60b3      	str	r3, [r6, #8]
 8000dd6:	e8bd 87f0 	ldmia.w	sp!, {r4, r5, r6, r7, r8, r9, sl, pc}
      huart->Instance->BRR = UART_BRR_SAMPLING8(HAL_RCC_GetPCLK1Freq(), huart->Init.BaudRate);
 8000dda:	f7ff ff71 	bl	8000cc0 <HAL_RCC_GetPCLK1Freq>
 8000dde:	2519      	movs	r5, #25
 8000de0:	fb05 f300 	mul.w	r3, r5, r0
 8000de4:	6860      	ldr	r0, [r4, #4]
 8000de6:	f04f 0964 	mov.w	r9, #100	; 0x64
 8000dea:	0040      	lsls	r0, r0, #1
 8000dec:	fbb3 f3f0 	udiv	r3, r3, r0
 8000df0:	fbb3 f3f9 	udiv	r3, r3, r9
 8000df4:	ea4f 1803 	mov.w	r8, r3, lsl #4
 8000df8:	f7ff ff62 	bl	8000cc0 <HAL_RCC_GetPCLK1Freq>
 8000dfc:	6863      	ldr	r3, [r4, #4]
 8000dfe:	4368      	muls	r0, r5
 8000e00:	005b      	lsls	r3, r3, #1
 8000e02:	fbb0 f7f3 	udiv	r7, r0, r3
 8000e06:	f7ff ff5b 	bl	8000cc0 <HAL_RCC_GetPCLK1Freq>
 8000e0a:	6863      	ldr	r3, [r4, #4]
 8000e0c:	4368      	muls	r0, r5
 8000e0e:	005b      	lsls	r3, r3, #1
 8000e10:	fbb0 f3f3 	udiv	r3, r0, r3
 8000e14:	fbb3 f3f9 	udiv	r3, r3, r9
 8000e18:	fb09 7313 	mls	r3, r9, r3, r7
 8000e1c:	00db      	lsls	r3, r3, #3
 8000e1e:	3332      	adds	r3, #50	; 0x32
 8000e20:	fbb3 f3f9 	udiv	r3, r3, r9
 8000e24:	005b      	lsls	r3, r3, #1
 8000e26:	f403 77f8 	and.w	r7, r3, #496	; 0x1f0
 8000e2a:	f7ff ff49 	bl	8000cc0 <HAL_RCC_GetPCLK1Freq>
 8000e2e:	6862      	ldr	r2, [r4, #4]
 8000e30:	4368      	muls	r0, r5
 8000e32:	0052      	lsls	r2, r2, #1
 8000e34:	fbb0 faf2 	udiv	sl, r0, r2
 8000e38:	f7ff ff42 	bl	8000cc0 <HAL_RCC_GetPCLK1Freq>
 8000e3c:	e7b9      	b.n	8000db2 <UART_SetConfig+0xb2>
    if ((huart->Instance == USART1) || (huart->Instance == USART6))
 8000e3e:	429e      	cmp	r6, r3
 8000e40:	d002      	beq.n	8000e48 <UART_SetConfig+0x148>
 8000e42:	4b3b      	ldr	r3, [pc, #236]	; (8000f30 <UART_SetConfig+0x230>)
 8000e44:	429e      	cmp	r6, r3
 8000e46:	d140      	bne.n	8000eca <UART_SetConfig+0x1ca>
      huart->Instance->BRR = UART_BRR_SAMPLING16(HAL_RCC_GetPCLK2Freq(), huart->Init.BaudRate);
 8000e48:	f7ff ff4a 	bl	8000ce0 <HAL_RCC_GetPCLK2Freq>
 8000e4c:	6867      	ldr	r7, [r4, #4]
 8000e4e:	2519      	movs	r5, #25
 8000e50:	f04f 0964 	mov.w	r9, #100	; 0x64
 8000e54:	fb05 f300 	mul.w	r3, r5, r0
 8000e58:	00bf      	lsls	r7, r7, #2
 8000e5a:	fbb3 f3f7 	udiv	r3, r3, r7
 8000e5e:	fbb3 f3f9 	udiv	r3, r3, r9
 8000e62:	011f      	lsls	r7, r3, #4
 8000e64:	f7ff ff3c 	bl	8000ce0 <HAL_RCC_GetPCLK2Freq>
 8000e68:	6863      	ldr	r3, [r4, #4]
 8000e6a:	4368      	muls	r0, r5
 8000e6c:	009b      	lsls	r3, r3, #2
 8000e6e:	fbb0 f8f3 	udiv	r8, r0, r3
 8000e72:	f7ff ff35 	bl	8000ce0 <HAL_RCC_GetPCLK2Freq>
 8000e76:	6863      	ldr	r3, [r4, #4]
 8000e78:	4368      	muls	r0, r5
 8000e7a:	009b      	lsls	r3, r3, #2
 8000e7c:	fbb0 f3f3 	udiv	r3, r0, r3
 8000e80:	fbb3 f3f9 	udiv	r3, r3, r9
 8000e84:	fb09 8313 	mls	r3, r9, r3, r8
 8000e88:	011b      	lsls	r3, r3, #4
 8000e8a:	3332      	adds	r3, #50	; 0x32
 8000e8c:	fbb3 f3f9 	udiv	r3, r3, r9
 8000e90:	f003 08f0 	and.w	r8, r3, #240	; 0xf0
 8000e94:	f7ff ff24 	bl	8000ce0 <HAL_RCC_GetPCLK2Freq>
 8000e98:	6862      	ldr	r2, [r4, #4]
 8000e9a:	4368      	muls	r0, r5
 8000e9c:	0092      	lsls	r2, r2, #2
 8000e9e:	fbb0 faf2 	udiv	sl, r0, r2
 8000ea2:	f7ff ff1d 	bl	8000ce0 <HAL_RCC_GetPCLK2Freq>
      huart->Instance->BRR = UART_BRR_SAMPLING16(HAL_RCC_GetPCLK1Freq(), huart->Init.BaudRate);
 8000ea6:	6863      	ldr	r3, [r4, #4]
 8000ea8:	4368      	muls	r0, r5
 8000eaa:	009b      	lsls	r3, r3, #2
 8000eac:	fbb0 f3f3 	udiv	r3, r0, r3
 8000eb0:	fbb3 f3f9 	udiv	r3, r3, r9
 8000eb4:	fb09 a313 	mls	r3, r9, r3, sl
 8000eb8:	011b      	lsls	r3, r3, #4
 8000eba:	3332      	adds	r3, #50	; 0x32
 8000ebc:	fbb3 f3f9 	udiv	r3, r3, r9
 8000ec0:	f003 030f 	and.w	r3, r3, #15
 8000ec4:	ea43 0308 	orr.w	r3, r3, r8
 8000ec8:	e783      	b.n	8000dd2 <UART_SetConfig+0xd2>
 8000eca:	f7ff fef9 	bl	8000cc0 <HAL_RCC_GetPCLK1Freq>
 8000ece:	6867      	ldr	r7, [r4, #4]
 8000ed0:	2519      	movs	r5, #25
 8000ed2:	f04f 0964 	mov.w	r9, #100	; 0x64
 8000ed6:	fb05 f300 	mul.w	r3, r5, r0
 8000eda:	00bf      	lsls	r7, r7, #2
 8000edc:	fbb3 f3f7 	udiv	r3, r3, r7
 8000ee0:	fbb3 f3f9 	udiv	r3, r3, r9
 8000ee4:	011f      	lsls	r7, r3, #4
 8000ee6:	f7ff feeb 	bl	8000cc0 <HAL_RCC_GetPCLK1Freq>
 8000eea:	6863      	ldr	r3, [r4, #4]
 8000eec:	4368      	muls	r0, r5
 8000eee:	009b      	lsls	r3, r3, #2
 8000ef0:	fbb0 f8f3 	udiv	r8, r0, r3
 8000ef4:	f7ff fee4 	bl	8000cc0 <HAL_RCC_GetPCLK1Freq>
 8000ef8:	6863      	ldr	r3, [r4, #4]
 8000efa:	4368      	muls	r0, r5
 8000efc:	009b      	lsls	r3, r3, #2
 8000efe:	fbb0 f3f3 	udiv	r3, r0, r3
 8000f02:	fbb3 f3f9 	udiv	r3, r3, r9
 8000f06:	fb09 8313 	mls	r3, r9, r3, r8
 8000f0a:	011b      	lsls	r3, r3, #4
 8000f0c:	3332      	adds	r3, #50	; 0x32
 8000f0e:	fbb3 f3f9 	udiv	r3, r3, r9
 8000f12:	f003 08f0 	and.w	r8, r3, #240	; 0xf0
 8000f16:	f7ff fed3 	bl	8000cc0 <HAL_RCC_GetPCLK1Freq>
 8000f1a:	6862      	ldr	r2, [r4, #4]
 8000f1c:	4368      	muls	r0, r5
 8000f1e:	0092      	lsls	r2, r2, #2
 8000f20:	fbb0 faf2 	udiv	sl, r0, r2
 8000f24:	f7ff fecc 	bl	8000cc0 <HAL_RCC_GetPCLK1Freq>
 8000f28:	e7bd      	b.n	8000ea6 <UART_SetConfig+0x1a6>
 8000f2a:	bf00      	nop
 8000f2c:	40011000 	.word	0x40011000
 8000f30:	40011400 	.word	0x40011400

08000f34 <HAL_UART_Init>:
{
 8000f34:	b510      	push	{r4, lr}
  if (huart == NULL)
 8000f36:	4604      	mov	r4, r0
 8000f38:	b340      	cbz	r0, 8000f8c <HAL_UART_Init+0x58>
  if (huart->gState == HAL_UART_STATE_RESET)
 8000f3a:	f890 3039 	ldrb.w	r3, [r0, #57]	; 0x39
 8000f3e:	f003 02ff 	and.w	r2, r3, #255	; 0xff
 8000f42:	b91b      	cbnz	r3, 8000f4c <HAL_UART_Init+0x18>
    huart->Lock = HAL_UNLOCKED;
 8000f44:	f880 2038 	strb.w	r2, [r0, #56]	; 0x38
    HAL_UART_MspInit(huart);
 8000f48:	f000 f8fe 	bl	8001148 <HAL_UART_MspInit>
  __HAL_UART_DISABLE(huart);
 8000f4c:	6822      	ldr	r2, [r4, #0]
  huart->gState = HAL_UART_STATE_BUSY;
 8000f4e:	2324      	movs	r3, #36	; 0x24
 8000f50:	f884 3039 	strb.w	r3, [r4, #57]	; 0x39
  __HAL_UART_DISABLE(huart);
 8000f54:	68d3      	ldr	r3, [r2, #12]
 8000f56:	f423 5300 	bic.w	r3, r3, #8192	; 0x2000
 8000f5a:	60d3      	str	r3, [r2, #12]
  UART_SetConfig(huart);
 8000f5c:	4620      	mov	r0, r4
 8000f5e:	f7ff fecf 	bl	8000d00 <UART_SetConfig>
  CLEAR_BIT(huart->Instance->CR2, (USART_CR2_LINEN | USART_CR2_CLKEN));
 8000f62:	6823      	ldr	r3, [r4, #0]
 8000f64:	691a      	ldr	r2, [r3, #16]
 8000f66:	f422 4290 	bic.w	r2, r2, #18432	; 0x4800
 8000f6a:	611a      	str	r2, [r3, #16]
  CLEAR_BIT(huart->Instance->CR3, (USART_CR3_SCEN | USART_CR3_HDSEL | USART_CR3_IREN));
 8000f6c:	695a      	ldr	r2, [r3, #20]
 8000f6e:	f022 022a 	bic.w	r2, r2, #42	; 0x2a
 8000f72:	615a      	str	r2, [r3, #20]
  __HAL_UART_ENABLE(huart);
 8000f74:	68da      	ldr	r2, [r3, #12]
 8000f76:	f442 5200 	orr.w	r2, r2, #8192	; 0x2000
 8000f7a:	60da      	str	r2, [r3, #12]
  huart->ErrorCode = HAL_UART_ERROR_NONE;
 8000f7c:	2000      	movs	r0, #0
  huart->gState = HAL_UART_STATE_READY;
 8000f7e:	2320      	movs	r3, #32
  huart->ErrorCode = HAL_UART_ERROR_NONE;
 8000f80:	63e0      	str	r0, [r4, #60]	; 0x3c
  huart->gState = HAL_UART_STATE_READY;
 8000f82:	f884 3039 	strb.w	r3, [r4, #57]	; 0x39
  huart->RxState = HAL_UART_STATE_READY;
 8000f86:	f884 303a 	strb.w	r3, [r4, #58]	; 0x3a
  return HAL_OK;
 8000f8a:	bd10      	pop	{r4, pc}
    return HAL_ERROR;
 8000f8c:	2001      	movs	r0, #1
}
 8000f8e:	bd10      	pop	{r4, pc}

08000f90 <SystemClock_Config>:
/**
  * @brief System Clock Configuration
  * @retval None
  */
void SystemClock_Config(void)
{
 8000f90:	b530      	push	{r4, r5, lr}
 8000f92:	b095      	sub	sp, #84	; 0x54
  RCC_OscInitTypeDef RCC_OscInitStruct = {0};
 8000f94:	2230      	movs	r2, #48	; 0x30
 8000f96:	2100      	movs	r1, #0
 8000f98:	a808      	add	r0, sp, #32
 8000f9a:	f000 f98b 	bl	80012b4 <memset>
  RCC_ClkInitTypeDef RCC_ClkInitStruct = {0};
 8000f9e:	2100      	movs	r1, #0
 8000fa0:	2214      	movs	r2, #20
 8000fa2:	a803      	add	r0, sp, #12
 8000fa4:	f000 f986 	bl	80012b4 <memset>

  /** Configure the main internal regulator output voltage 
  */
  __HAL_RCC_PWR_CLK_ENABLE();
 8000fa8:	2400      	movs	r4, #0
 8000faa:	4b1b      	ldr	r3, [pc, #108]	; (8001018 <SystemClock_Config+0x88>)
 8000fac:	9401      	str	r4, [sp, #4]
 8000fae:	6c1a      	ldr	r2, [r3, #64]	; 0x40
 8000fb0:	f042 5280 	orr.w	r2, r2, #268435456	; 0x10000000
 8000fb4:	641a      	str	r2, [r3, #64]	; 0x40
 8000fb6:	6c1b      	ldr	r3, [r3, #64]	; 0x40
 8000fb8:	f003 5380 	and.w	r3, r3, #268435456	; 0x10000000
 8000fbc:	9301      	str	r3, [sp, #4]
 8000fbe:	9b01      	ldr	r3, [sp, #4]
  __HAL_PWR_VOLTAGESCALING_CONFIG(PWR_REGULATOR_VOLTAGE_SCALE1);
 8000fc0:	4b16      	ldr	r3, [pc, #88]	; (800101c <SystemClock_Config+0x8c>)
 8000fc2:	9402      	str	r4, [sp, #8]
 8000fc4:	681a      	ldr	r2, [r3, #0]
 8000fc6:	f442 4240 	orr.w	r2, r2, #49152	; 0xc000
 8000fca:	601a      	str	r2, [r3, #0]
 8000fcc:	681b      	ldr	r3, [r3, #0]
  */
  RCC_OscInitStruct.OscillatorType = RCC_OSCILLATORTYPE_HSI;
  RCC_OscInitStruct.HSIState = RCC_HSI_ON;
  RCC_OscInitStruct.HSICalibrationValue = RCC_HSICALIBRATION_DEFAULT;
  RCC_OscInitStruct.PLL.PLLState = RCC_PLL_ON;
  RCC_OscInitStruct.PLL.PLLSource = RCC_PLLSOURCE_HSI;
 8000fce:	940f      	str	r4, [sp, #60]	; 0x3c
  __HAL_PWR_VOLTAGESCALING_CONFIG(PWR_REGULATOR_VOLTAGE_SCALE1);
 8000fd0:	f403 4340 	and.w	r3, r3, #49152	; 0xc000
 8000fd4:	9302      	str	r3, [sp, #8]
 8000fd6:	9b02      	ldr	r3, [sp, #8]
  RCC_OscInitStruct.HSIState = RCC_HSI_ON;
 8000fd8:	2301      	movs	r3, #1
 8000fda:	930b      	str	r3, [sp, #44]	; 0x2c
  RCC_OscInitStruct.HSICalibrationValue = RCC_HSICALIBRATION_DEFAULT;
 8000fdc:	2310      	movs	r3, #16
 8000fde:	930c      	str	r3, [sp, #48]	; 0x30
  RCC_OscInitStruct.PLL.PLLM = 8;
 8000fe0:	2308      	movs	r3, #8
 8000fe2:	9310      	str	r3, [sp, #64]	; 0x40
  RCC_OscInitStruct.PLL.PLLN = 100;
 8000fe4:	2364      	movs	r3, #100	; 0x64
  RCC_OscInitStruct.OscillatorType = RCC_OSCILLATORTYPE_HSI;
 8000fe6:	2502      	movs	r5, #2
  RCC_OscInitStruct.PLL.PLLN = 100;
 8000fe8:	9311      	str	r3, [sp, #68]	; 0x44
  RCC_OscInitStruct.PLL.PLLP = RCC_PLLP_DIV2;
  RCC_OscInitStruct.PLL.PLLQ = 4;
  if (HAL_RCC_OscConfig(&RCC_OscInitStruct) != HAL_OK)
 8000fea:	a808      	add	r0, sp, #32
  RCC_OscInitStruct.PLL.PLLQ = 4;
 8000fec:	2304      	movs	r3, #4
 8000fee:	9313      	str	r3, [sp, #76]	; 0x4c
  RCC_OscInitStruct.OscillatorType = RCC_OSCILLATORTYPE_HSI;
 8000ff0:	9508      	str	r5, [sp, #32]
  RCC_OscInitStruct.PLL.PLLState = RCC_PLL_ON;
 8000ff2:	950e      	str	r5, [sp, #56]	; 0x38
  RCC_OscInitStruct.PLL.PLLP = RCC_PLLP_DIV2;
 8000ff4:	9512      	str	r5, [sp, #72]	; 0x48
  if (HAL_RCC_OscConfig(&RCC_OscInitStruct) != HAL_OK)
 8000ff6:	f7ff fc19 	bl	800082c <HAL_RCC_OscConfig>
  {
    Error_Handler();
  }
  /** Initializes the CPU, AHB and APB busses clocks 
  */
  RCC_ClkInitStruct.ClockType = RCC_CLOCKTYPE_HCLK|RCC_CLOCKTYPE_SYSCLK
 8000ffa:	230f      	movs	r3, #15
 8000ffc:	9303      	str	r3, [sp, #12]
  RCC_ClkInitStruct.SYSCLKSource = RCC_SYSCLKSOURCE_PLLCLK;
  RCC_ClkInitStruct.AHBCLKDivider = RCC_SYSCLK_DIV1;
  RCC_ClkInitStruct.APB1CLKDivider = RCC_HCLK_DIV2;
  RCC_ClkInitStruct.APB2CLKDivider = RCC_HCLK_DIV1;

  if (HAL_RCC_ClockConfig(&RCC_ClkInitStruct, FLASH_LATENCY_3) != HAL_OK)
 8000ffe:	2103      	movs	r1, #3
  RCC_ClkInitStruct.APB1CLKDivider = RCC_HCLK_DIV2;
 8001000:	f44f 5380 	mov.w	r3, #4096	; 0x1000
  if (HAL_RCC_ClockConfig(&RCC_ClkInitStruct, FLASH_LATENCY_3) != HAL_OK)
 8001004:	a803      	add	r0, sp, #12
  RCC_ClkInitStruct.SYSCLKSource = RCC_SYSCLKSOURCE_PLLCLK;
 8001006:	9504      	str	r5, [sp, #16]
  RCC_ClkInitStruct.AHBCLKDivider = RCC_SYSCLK_DIV1;
 8001008:	9405      	str	r4, [sp, #20]
  RCC_ClkInitStruct.APB1CLKDivider = RCC_HCLK_DIV2;
 800100a:	9306      	str	r3, [sp, #24]
  RCC_ClkInitStruct.APB2CLKDivider = RCC_HCLK_DIV1;
 800100c:	9407      	str	r4, [sp, #28]
  if (HAL_RCC_ClockConfig(&RCC_ClkInitStruct, FLASH_LATENCY_3) != HAL_OK)
 800100e:	f7ff fdbd 	bl	8000b8c <HAL_RCC_ClockConfig>
  {
    Error_Handler();
  }
}
 8001012:	b015      	add	sp, #84	; 0x54
 8001014:	bd30      	pop	{r4, r5, pc}
 8001016:	bf00      	nop
 8001018:	40023800 	.word	0x40023800
 800101c:	40007000 	.word	0x40007000

08001020 <main>:
{
 8001020:	b500      	push	{lr}
 8001022:	b08b      	sub	sp, #44	; 0x2c
  HAL_Init();
 8001024:	f7ff fa84 	bl	8000530 <HAL_Init>
  SystemClock_Config();
 8001028:	f7ff ffb2 	bl	8000f90 <SystemClock_Config>
  * @param None
  * @retval None
  */
static void MX_GPIO_Init(void)
{
  GPIO_InitTypeDef GPIO_InitStruct = {0};
 800102c:	2214      	movs	r2, #20
 800102e:	2100      	movs	r1, #0
 8001030:	eb0d 0002 	add.w	r0, sp, r2
 8001034:	f000 f93e 	bl	80012b4 <memset>

  /* GPIO Ports Clock Enable */
  __HAL_RCC_GPIOC_CLK_ENABLE();
 8001038:	2400      	movs	r4, #0
 800103a:	4b2d      	ldr	r3, [pc, #180]	; (80010f0 <main+0xd0>)
 800103c:	9401      	str	r4, [sp, #4]
 800103e:	6b1a      	ldr	r2, [r3, #48]	; 0x30
  __HAL_RCC_GPIOH_CLK_ENABLE();
  __HAL_RCC_GPIOA_CLK_ENABLE();
  __HAL_RCC_GPIOB_CLK_ENABLE();

  /*Configure GPIO pin Output Level */
  HAL_GPIO_WritePin(LD2_GPIO_Port, LD2_Pin, GPIO_PIN_RESET);
 8001040:	482c      	ldr	r0, [pc, #176]	; (80010f4 <main+0xd4>)
  __HAL_RCC_GPIOC_CLK_ENABLE();
 8001042:	f042 0204 	orr.w	r2, r2, #4
 8001046:	631a      	str	r2, [r3, #48]	; 0x30
 8001048:	6b1a      	ldr	r2, [r3, #48]	; 0x30
 800104a:	f002 0204 	and.w	r2, r2, #4
 800104e:	9201      	str	r2, [sp, #4]
 8001050:	9a01      	ldr	r2, [sp, #4]
  __HAL_RCC_GPIOH_CLK_ENABLE();
 8001052:	9402      	str	r4, [sp, #8]
 8001054:	6b1a      	ldr	r2, [r3, #48]	; 0x30
 8001056:	f042 0280 	orr.w	r2, r2, #128	; 0x80
 800105a:	631a      	str	r2, [r3, #48]	; 0x30
 800105c:	6b1a      	ldr	r2, [r3, #48]	; 0x30
 800105e:	f002 0280 	and.w	r2, r2, #128	; 0x80
 8001062:	9202      	str	r2, [sp, #8]
 8001064:	9a02      	ldr	r2, [sp, #8]
  __HAL_RCC_GPIOA_CLK_ENABLE();
 8001066:	9403      	str	r4, [sp, #12]
 8001068:	6b1a      	ldr	r2, [r3, #48]	; 0x30
 800106a:	f042 0201 	orr.w	r2, r2, #1
 800106e:	631a      	str	r2, [r3, #48]	; 0x30
 8001070:	6b1a      	ldr	r2, [r3, #48]	; 0x30
 8001072:	f002 0201 	and.w	r2, r2, #1
 8001076:	9203      	str	r2, [sp, #12]
 8001078:	9a03      	ldr	r2, [sp, #12]
  __HAL_RCC_GPIOB_CLK_ENABLE();
 800107a:	9404      	str	r4, [sp, #16]
 800107c:	6b1a      	ldr	r2, [r3, #48]	; 0x30
 800107e:	f042 0202 	orr.w	r2, r2, #2
 8001082:	631a      	str	r2, [r3, #48]	; 0x30
 8001084:	6b1b      	ldr	r3, [r3, #48]	; 0x30
 8001086:	f003 0302 	and.w	r3, r3, #2
  HAL_GPIO_WritePin(LD2_GPIO_Port, LD2_Pin, GPIO_PIN_RESET);
 800108a:	4622      	mov	r2, r4
  __HAL_RCC_GPIOB_CLK_ENABLE();
 800108c:	9304      	str	r3, [sp, #16]
  HAL_GPIO_WritePin(LD2_GPIO_Port, LD2_Pin, GPIO_PIN_RESET);
 800108e:	2120      	movs	r1, #32
  __HAL_RCC_GPIOB_CLK_ENABLE();
 8001090:	9b04      	ldr	r3, [sp, #16]
  HAL_GPIO_WritePin(LD2_GPIO_Port, LD2_Pin, GPIO_PIN_RESET);
 8001092:	f7ff fbbf 	bl	8000814 <HAL_GPIO_WritePin>

  /*Configure GPIO pin : B1_Pin */
  GPIO_InitStruct.Pin = B1_Pin;
 8001096:	f44f 5300 	mov.w	r3, #8192	; 0x2000
 800109a:	9305      	str	r3, [sp, #20]
  GPIO_InitStruct.Mode = GPIO_MODE_IT_FALLING;
  GPIO_InitStruct.Pull = GPIO_NOPULL;
  HAL_GPIO_Init(B1_GPIO_Port, &GPIO_InitStruct);
 800109c:	a905      	add	r1, sp, #20
  GPIO_InitStruct.Mode = GPIO_MODE_IT_FALLING;
 800109e:	4b16      	ldr	r3, [pc, #88]	; (80010f8 <main+0xd8>)
  HAL_GPIO_Init(B1_GPIO_Port, &GPIO_InitStruct);
 80010a0:	4816      	ldr	r0, [pc, #88]	; (80010fc <main+0xdc>)
  GPIO_InitStruct.Mode = GPIO_MODE_IT_FALLING;
 80010a2:	9306      	str	r3, [sp, #24]
  GPIO_InitStruct.Pull = GPIO_NOPULL;
 80010a4:	9407      	str	r4, [sp, #28]
  HAL_GPIO_Init(B1_GPIO_Port, &GPIO_InitStruct);
 80010a6:	f7ff fadf 	bl	8000668 <HAL_GPIO_Init>

  /*Configure GPIO pin : LD2_Pin */
  GPIO_InitStruct.Pin = LD2_Pin;
 80010aa:	2320      	movs	r3, #32
 80010ac:	9305      	str	r3, [sp, #20]
  GPIO_InitStruct.Mode = GPIO_MODE_OUTPUT_PP;
  GPIO_InitStruct.Pull = GPIO_NOPULL;
  GPIO_InitStruct.Speed = GPIO_SPEED_FREQ_LOW;
  HAL_GPIO_Init(LD2_GPIO_Port, &GPIO_InitStruct);
 80010ae:	a905      	add	r1, sp, #20
  GPIO_InitStruct.Mode = GPIO_MODE_OUTPUT_PP;
 80010b0:	2301      	movs	r3, #1
  HAL_GPIO_Init(LD2_GPIO_Port, &GPIO_InitStruct);
 80010b2:	4810      	ldr	r0, [pc, #64]	; (80010f4 <main+0xd4>)
  GPIO_InitStruct.Mode = GPIO_MODE_OUTPUT_PP;
 80010b4:	9306      	str	r3, [sp, #24]
  GPIO_InitStruct.Pull = GPIO_NOPULL;
 80010b6:	9407      	str	r4, [sp, #28]
  GPIO_InitStruct.Speed = GPIO_SPEED_FREQ_LOW;
 80010b8:	9408      	str	r4, [sp, #32]
  HAL_GPIO_Init(LD2_GPIO_Port, &GPIO_InitStruct);
 80010ba:	f7ff fad5 	bl	8000668 <HAL_GPIO_Init>
  huart2.Instance = USART2;
 80010be:	4810      	ldr	r0, [pc, #64]	; (8001100 <main+0xe0>)
  huart2.Init.BaudRate = 115200;
 80010c0:	4a10      	ldr	r2, [pc, #64]	; (8001104 <main+0xe4>)
  huart2.Init.WordLength = UART_WORDLENGTH_8B;
 80010c2:	6084      	str	r4, [r0, #8]
  huart2.Init.BaudRate = 115200;
 80010c4:	f44f 33e1 	mov.w	r3, #115200	; 0x1c200
 80010c8:	e880 000c 	stmia.w	r0, {r2, r3}
  huart2.Init.Mode = UART_MODE_TX_RX;
 80010cc:	230c      	movs	r3, #12
  huart2.Init.StopBits = UART_STOPBITS_1;
 80010ce:	60c4      	str	r4, [r0, #12]
  huart2.Init.Parity = UART_PARITY_NONE;
 80010d0:	6104      	str	r4, [r0, #16]
  huart2.Init.HwFlowCtl = UART_HWCONTROL_NONE;
 80010d2:	6184      	str	r4, [r0, #24]
  huart2.Init.OverSampling = UART_OVERSAMPLING_16;
 80010d4:	61c4      	str	r4, [r0, #28]
  huart2.Init.Mode = UART_MODE_TX_RX;
 80010d6:	6143      	str	r3, [r0, #20]
  if (HAL_UART_Init(&huart2) != HAL_OK)
 80010d8:	f7ff ff2c 	bl	8000f34 <HAL_UART_Init>
	  HAL_GPIO_TogglePin(LD2_GPIO_Port,LD2_Pin);
 80010dc:	4c05      	ldr	r4, [pc, #20]	; (80010f4 <main+0xd4>)
 80010de:	4620      	mov	r0, r4
 80010e0:	2120      	movs	r1, #32
 80010e2:	f7ff fb9c 	bl	800081e <HAL_GPIO_TogglePin>
	  HAL_Delay(200);
 80010e6:	20c8      	movs	r0, #200	; 0xc8
 80010e8:	f7ff fa4e 	bl	8000588 <HAL_Delay>
 80010ec:	e7f7      	b.n	80010de <main+0xbe>
 80010ee:	bf00      	nop
 80010f0:	40023800 	.word	0x40023800
 80010f4:	40020000 	.word	0x40020000
 80010f8:	10210000 	.word	0x10210000
 80010fc:	40020800 	.word	0x40020800
 8001100:	2000002c 	.word	0x2000002c
 8001104:	40004400 	.word	0x40004400

08001108 <HAL_MspInit>:
/* USER CODE END 0 */
/**
  * Initializes the Global MSP.
  */
void HAL_MspInit(void)
{
 8001108:	b507      	push	{r0, r1, r2, lr}
  /* USER CODE BEGIN MspInit 0 */

  /* USER CODE END MspInit 0 */

  __HAL_RCC_SYSCFG_CLK_ENABLE();
 800110a:	4b0e      	ldr	r3, [pc, #56]	; (8001144 <HAL_MspInit+0x3c>)
 800110c:	2100      	movs	r1, #0
 800110e:	9100      	str	r1, [sp, #0]
 8001110:	6c5a      	ldr	r2, [r3, #68]	; 0x44
 8001112:	f442 4280 	orr.w	r2, r2, #16384	; 0x4000
 8001116:	645a      	str	r2, [r3, #68]	; 0x44
 8001118:	6c5a      	ldr	r2, [r3, #68]	; 0x44
 800111a:	f402 4280 	and.w	r2, r2, #16384	; 0x4000
 800111e:	9200      	str	r2, [sp, #0]
 8001120:	9a00      	ldr	r2, [sp, #0]
  __HAL_RCC_PWR_CLK_ENABLE();
 8001122:	9101      	str	r1, [sp, #4]
 8001124:	6c1a      	ldr	r2, [r3, #64]	; 0x40
 8001126:	f042 5280 	orr.w	r2, r2, #268435456	; 0x10000000
 800112a:	641a      	str	r2, [r3, #64]	; 0x40
 800112c:	6c1b      	ldr	r3, [r3, #64]	; 0x40
 800112e:	f003 5380 	and.w	r3, r3, #268435456	; 0x10000000
 8001132:	9301      	str	r3, [sp, #4]

  HAL_NVIC_SetPriorityGrouping(NVIC_PRIORITYGROUP_0);
 8001134:	2007      	movs	r0, #7
  __HAL_RCC_PWR_CLK_ENABLE();
 8001136:	9b01      	ldr	r3, [sp, #4]
  HAL_NVIC_SetPriorityGrouping(NVIC_PRIORITYGROUP_0);
 8001138:	f7ff fa3a 	bl	80005b0 <HAL_NVIC_SetPriorityGrouping>
  /* System interrupt init*/

  /* USER CODE BEGIN MspInit 1 */

  /* USER CODE END MspInit 1 */
}
 800113c:	b003      	add	sp, #12
 800113e:	f85d fb04 	ldr.w	pc, [sp], #4
 8001142:	bf00      	nop
 8001144:	40023800 	.word	0x40023800

08001148 <HAL_UART_MspInit>:
* This function configures the hardware resources used in this example
* @param huart: UART handle pointer
* @retval None
*/
void HAL_UART_MspInit(UART_HandleTypeDef* huart)
{
 8001148:	b510      	push	{r4, lr}
 800114a:	4604      	mov	r4, r0
 800114c:	b088      	sub	sp, #32
  GPIO_InitTypeDef GPIO_InitStruct = {0};
 800114e:	2214      	movs	r2, #20
 8001150:	2100      	movs	r1, #0
 8001152:	a803      	add	r0, sp, #12
 8001154:	f000 f8ae 	bl	80012b4 <memset>
  if(huart->Instance==USART2)
 8001158:	6822      	ldr	r2, [r4, #0]
 800115a:	4b15      	ldr	r3, [pc, #84]	; (80011b0 <HAL_UART_MspInit+0x68>)
 800115c:	429a      	cmp	r2, r3
 800115e:	d124      	bne.n	80011aa <HAL_UART_MspInit+0x62>
  {
  /* USER CODE BEGIN USART2_MspInit 0 */

  /* USER CODE END USART2_MspInit 0 */
    /* Peripheral clock enable */
    __HAL_RCC_USART2_CLK_ENABLE();
 8001160:	f503 33fa 	add.w	r3, r3, #128000	; 0x1f400
 8001164:	2100      	movs	r1, #0
 8001166:	9101      	str	r1, [sp, #4]
 8001168:	6c1a      	ldr	r2, [r3, #64]	; 0x40
    GPIO_InitStruct.Pin = USART_TX_Pin|USART_RX_Pin;
    GPIO_InitStruct.Mode = GPIO_MODE_AF_PP;
    GPIO_InitStruct.Pull = GPIO_PULLUP;
    GPIO_InitStruct.Speed = GPIO_SPEED_FREQ_VERY_HIGH;
    GPIO_InitStruct.Alternate = GPIO_AF7_USART2;
    HAL_GPIO_Init(GPIOA, &GPIO_InitStruct);
 800116a:	4812      	ldr	r0, [pc, #72]	; (80011b4 <HAL_UART_MspInit+0x6c>)
    __HAL_RCC_USART2_CLK_ENABLE();
 800116c:	f442 3200 	orr.w	r2, r2, #131072	; 0x20000
 8001170:	641a      	str	r2, [r3, #64]	; 0x40
 8001172:	6c1a      	ldr	r2, [r3, #64]	; 0x40
 8001174:	f402 3200 	and.w	r2, r2, #131072	; 0x20000
 8001178:	9201      	str	r2, [sp, #4]
 800117a:	9a01      	ldr	r2, [sp, #4]
    __HAL_RCC_GPIOA_CLK_ENABLE();
 800117c:	9102      	str	r1, [sp, #8]
 800117e:	6b1a      	ldr	r2, [r3, #48]	; 0x30
 8001180:	f042 0201 	orr.w	r2, r2, #1
 8001184:	631a      	str	r2, [r3, #48]	; 0x30
 8001186:	6b1b      	ldr	r3, [r3, #48]	; 0x30
 8001188:	f003 0301 	and.w	r3, r3, #1
 800118c:	9302      	str	r3, [sp, #8]
 800118e:	9b02      	ldr	r3, [sp, #8]
    GPIO_InitStruct.Pin = USART_TX_Pin|USART_RX_Pin;
 8001190:	230c      	movs	r3, #12
 8001192:	9303      	str	r3, [sp, #12]
    GPIO_InitStruct.Mode = GPIO_MODE_AF_PP;
 8001194:	2302      	movs	r3, #2
 8001196:	9304      	str	r3, [sp, #16]
    GPIO_InitStruct.Pull = GPIO_PULLUP;
 8001198:	2301      	movs	r3, #1
 800119a:	9305      	str	r3, [sp, #20]
    GPIO_InitStruct.Speed = GPIO_SPEED_FREQ_VERY_HIGH;
 800119c:	2303      	movs	r3, #3
 800119e:	9306      	str	r3, [sp, #24]
    HAL_GPIO_Init(GPIOA, &GPIO_InitStruct);
 80011a0:	a903      	add	r1, sp, #12
    GPIO_InitStruct.Alternate = GPIO_AF7_USART2;
 80011a2:	2307      	movs	r3, #7
 80011a4:	9307      	str	r3, [sp, #28]
    HAL_GPIO_Init(GPIOA, &GPIO_InitStruct);
 80011a6:	f7ff fa5f 	bl	8000668 <HAL_GPIO_Init>
  /* USER CODE BEGIN USART2_MspInit 1 */

  /* USER CODE END USART2_MspInit 1 */
  }

}
 80011aa:	b008      	add	sp, #32
 80011ac:	bd10      	pop	{r4, pc}
 80011ae:	bf00      	nop
 80011b0:	40004400 	.word	0x40004400
 80011b4:	40020000 	.word	0x40020000

080011b8 <NMI_Handler>:
 80011b8:	4770      	bx	lr

080011ba <HardFault_Handler>:

/**
  * @brief This function handles Hard fault interrupt.
  */
void HardFault_Handler(void)
{
 80011ba:	e7fe      	b.n	80011ba <HardFault_Handler>

080011bc <MemManage_Handler>:

/**
  * @brief This function handles Memory management fault.
  */
void MemManage_Handler(void)
{
 80011bc:	e7fe      	b.n	80011bc <MemManage_Handler>

080011be <BusFault_Handler>:

/**
  * @brief This function handles Pre-fetch fault, memory access fault.
  */
void BusFault_Handler(void)
{
 80011be:	e7fe      	b.n	80011be <BusFault_Handler>

080011c0 <UsageFault_Handler>:

/**
  * @brief This function handles Undefined instruction or illegal state.
  */
void UsageFault_Handler(void)
{
 80011c0:	e7fe      	b.n	80011c0 <UsageFault_Handler>

080011c2 <SVC_Handler>:
 80011c2:	4770      	bx	lr

080011c4 <DebugMon_Handler>:
 80011c4:	4770      	bx	lr

080011c6 <PendSV_Handler>:

/**
  * @brief This function handles Pendable request for system service.
  */
void PendSV_Handler(void)
{
 80011c6:	4770      	bx	lr

080011c8 <SysTick_Handler>:
void SysTick_Handler(void)
{
  /* USER CODE BEGIN SysTick_IRQn 0 */

  /* USER CODE END SysTick_IRQn 0 */
  HAL_IncTick();
 80011c8:	f7ff b9cc 	b.w	8000564 <HAL_IncTick>

080011cc <SystemInit>:
  */
void SystemInit(void)
{
  /* FPU settings ------------------------------------------------------------*/
  #if (__FPU_PRESENT == 1) && (__FPU_USED == 1)
    SCB->CPACR |= ((3UL << 10*2)|(3UL << 11*2));  /* set CP10 and CP11 Full Access */
 80011cc:	490f      	ldr	r1, [pc, #60]	; (800120c <SystemInit+0x40>)
 80011ce:	f8d1 3088 	ldr.w	r3, [r1, #136]	; 0x88
 80011d2:	f443 0370 	orr.w	r3, r3, #15728640	; 0xf00000
 80011d6:	f8c1 3088 	str.w	r3, [r1, #136]	; 0x88
  #endif
  /* Reset the RCC clock configuration to the default reset state ------------*/
  /* Set HSION bit */
  RCC->CR |= (uint32_t)0x00000001;
 80011da:	4b0d      	ldr	r3, [pc, #52]	; (8001210 <SystemInit+0x44>)
 80011dc:	681a      	ldr	r2, [r3, #0]

  /* Reset CFGR register */
  RCC->CFGR = 0x00000000;
 80011de:	2000      	movs	r0, #0
  RCC->CR |= (uint32_t)0x00000001;
 80011e0:	f042 0201 	orr.w	r2, r2, #1
 80011e4:	601a      	str	r2, [r3, #0]
  RCC->CFGR = 0x00000000;
 80011e6:	6098      	str	r0, [r3, #8]

  /* Reset HSEON, CSSON and PLLON bits */
  RCC->CR &= (uint32_t)0xFEF6FFFF;
 80011e8:	681a      	ldr	r2, [r3, #0]
 80011ea:	f022 7284 	bic.w	r2, r2, #17301504	; 0x1080000
 80011ee:	f422 3280 	bic.w	r2, r2, #65536	; 0x10000
 80011f2:	601a      	str	r2, [r3, #0]

  /* Reset PLLCFGR register */
  RCC->PLLCFGR = 0x24003010;
 80011f4:	4a07      	ldr	r2, [pc, #28]	; (8001214 <SystemInit+0x48>)
 80011f6:	605a      	str	r2, [r3, #4]

  /* Reset HSEBYP bit */
  RCC->CR &= (uint32_t)0xFFFBFFFF;
 80011f8:	681a      	ldr	r2, [r3, #0]
 80011fa:	f422 2280 	bic.w	r2, r2, #262144	; 0x40000
 80011fe:	601a      	str	r2, [r3, #0]

  /* Disable all interrupts */
  RCC->CIR = 0x00000000;
 8001200:	60d8      	str	r0, [r3, #12]

  /* Configure the Vector Table location add offset address ------------------*/
#ifdef VECT_TAB_SRAM
  SCB->VTOR = SRAM_BASE | VECT_TAB_OFFSET; /* Vector Table Relocation in Internal SRAM */
#else
  SCB->VTOR = FLASH_BASE | VECT_TAB_OFFSET; /* Vector Table Relocation in Internal FLASH */
 8001202:	f04f 6300 	mov.w	r3, #134217728	; 0x8000000
 8001206:	608b      	str	r3, [r1, #8]
 8001208:	4770      	bx	lr
 800120a:	bf00      	nop
 800120c:	e000ed00 	.word	0xe000ed00
 8001210:	40023800 	.word	0x40023800
 8001214:	24003010 	.word	0x24003010

08001218 <Reset_Handler>:

    .section  .text.Reset_Handler
  .weak  Reset_Handler
  .type  Reset_Handler, %function
Reset_Handler:  
  ldr   sp, =_estack    		 /* set stack pointer */
 8001218:	f8df d034 	ldr.w	sp, [pc, #52]	; 8001250 <LoopFillZerobss+0x14>

/* Copy the data segment initializers from flash to SRAM */  
  movs  r1, #0
 800121c:	2100      	movs	r1, #0
  b  LoopCopyDataInit
 800121e:	e003      	b.n	8001228 <LoopCopyDataInit>

08001220 <CopyDataInit>:

CopyDataInit:
  ldr  r3, =_sidata
 8001220:	4b0c      	ldr	r3, [pc, #48]	; (8001254 <LoopFillZerobss+0x18>)
  ldr  r3, [r3, r1]
 8001222:	585b      	ldr	r3, [r3, r1]
  str  r3, [r0, r1]
 8001224:	5043      	str	r3, [r0, r1]
  adds  r1, r1, #4
 8001226:	3104      	adds	r1, #4

08001228 <LoopCopyDataInit>:
    
LoopCopyDataInit:
  ldr  r0, =_sdata
 8001228:	480b      	ldr	r0, [pc, #44]	; (8001258 <LoopFillZerobss+0x1c>)
  ldr  r3, =_edata
 800122a:	4b0c      	ldr	r3, [pc, #48]	; (800125c <LoopFillZerobss+0x20>)
  adds  r2, r0, r1
 800122c:	1842      	adds	r2, r0, r1
  cmp  r2, r3
 800122e:	429a      	cmp	r2, r3
  bcc  CopyDataInit
 8001230:	d3f6      	bcc.n	8001220 <CopyDataInit>
  ldr  r2, =_sbss
 8001232:	4a0b      	ldr	r2, [pc, #44]	; (8001260 <LoopFillZerobss+0x24>)
  b  LoopFillZerobss
 8001234:	e002      	b.n	800123c <LoopFillZerobss>

08001236 <FillZerobss>:
/* Zero fill the bss segment. */  
FillZerobss:
  movs  r3, #0
 8001236:	2300      	movs	r3, #0
  str  r3, [r2], #4
 8001238:	f842 3b04 	str.w	r3, [r2], #4

0800123c <LoopFillZerobss>:
    
LoopFillZerobss:
  ldr  r3, = _ebss
 800123c:	4b09      	ldr	r3, [pc, #36]	; (8001264 <LoopFillZerobss+0x28>)
  cmp  r2, r3
 800123e:	429a      	cmp	r2, r3
  bcc  FillZerobss
 8001240:	d3f9      	bcc.n	8001236 <FillZerobss>

/* Call the clock system intitialization function.*/
  bl  SystemInit   
 8001242:	f7ff ffc3 	bl	80011cc <SystemInit>
/* Call static constructors */
    bl __libc_init_array
 8001246:	f000 f811 	bl	800126c <__libc_init_array>
/* Call the application's entry point.*/
  bl  main
 800124a:	f7ff fee9 	bl	8001020 <main>
  bx  lr    
 800124e:	4770      	bx	lr
  ldr   sp, =_estack    		 /* set stack pointer */
 8001250:	20020000 	.word	0x20020000
  ldr  r3, =_sidata
 8001254:	08001304 	.word	0x08001304
  ldr  r0, =_sdata
 8001258:	20000000 	.word	0x20000000
  ldr  r3, =_edata
 800125c:	2000000c 	.word	0x2000000c
  ldr  r2, =_sbss
 8001260:	2000000c 	.word	0x2000000c
  ldr  r3, = _ebss
 8001264:	2000006c 	.word	0x2000006c

08001268 <ADC_IRQHandler>:
 * @retval None       
*/
    .section  .text.Default_Handler,"ax",%progbits
Default_Handler:
Infinite_Loop:
  b  Infinite_Loop
 8001268:	e7fe      	b.n	8001268 <ADC_IRQHandler>
	...

0800126c <__libc_init_array>:
 800126c:	b570      	push	{r4, r5, r6, lr}
 800126e:	4e0d      	ldr	r6, [pc, #52]	; (80012a4 <__libc_init_array+0x38>)
 8001270:	4c0d      	ldr	r4, [pc, #52]	; (80012a8 <__libc_init_array+0x3c>)
 8001272:	1ba4      	subs	r4, r4, r6
 8001274:	10a4      	asrs	r4, r4, #2
 8001276:	2500      	movs	r5, #0
 8001278:	42a5      	cmp	r5, r4
 800127a:	d109      	bne.n	8001290 <__libc_init_array+0x24>
 800127c:	4e0b      	ldr	r6, [pc, #44]	; (80012ac <__libc_init_array+0x40>)
 800127e:	4c0c      	ldr	r4, [pc, #48]	; (80012b0 <__libc_init_array+0x44>)
 8001280:	f000 f820 	bl	80012c4 <_init>
 8001284:	1ba4      	subs	r4, r4, r6
 8001286:	10a4      	asrs	r4, r4, #2
 8001288:	2500      	movs	r5, #0
 800128a:	42a5      	cmp	r5, r4
 800128c:	d105      	bne.n	800129a <__libc_init_array+0x2e>
 800128e:	bd70      	pop	{r4, r5, r6, pc}
 8001290:	f856 3025 	ldr.w	r3, [r6, r5, lsl #2]
 8001294:	4798      	blx	r3
 8001296:	3501      	adds	r5, #1
 8001298:	e7ee      	b.n	8001278 <__libc_init_array+0xc>
 800129a:	f856 3025 	ldr.w	r3, [r6, r5, lsl #2]
 800129e:	4798      	blx	r3
 80012a0:	3501      	adds	r5, #1
 80012a2:	e7f2      	b.n	800128a <__libc_init_array+0x1e>
 80012a4:	080012fc 	.word	0x080012fc
 80012a8:	080012fc 	.word	0x080012fc
 80012ac:	080012fc 	.word	0x080012fc
 80012b0:	08001300 	.word	0x08001300

080012b4 <memset>:
 80012b4:	4402      	add	r2, r0
 80012b6:	4603      	mov	r3, r0
 80012b8:	4293      	cmp	r3, r2
 80012ba:	d100      	bne.n	80012be <memset+0xa>
 80012bc:	4770      	bx	lr
 80012be:	f803 1b01 	strb.w	r1, [r3], #1
 80012c2:	e7f9      	b.n	80012b8 <memset+0x4>

080012c4 <_init>:
 80012c4:	b5f8      	push	{r3, r4, r5, r6, r7, lr}
 80012c6:	bf00      	nop
 80012c8:	bcf8      	pop	{r3, r4, r5, r6, r7}
 80012ca:	bc08      	pop	{r3}
 80012cc:	469e      	mov	lr, r3
 80012ce:	4770      	bx	lr

080012d0 <_fini>:
 80012d0:	b5f8      	push	{r3, r4, r5, r6, r7, lr}
 80012d2:	bf00      	nop
 80012d4:	bcf8      	pop	{r3, r4, r5, r6, r7}
 80012d6:	bc08      	pop	{r3}
 80012d8:	469e      	mov	lr, r3
 80012da:	4770      	bx	lr
